:0400000044EF10F0C9
:08000800046ED8CF05F0E0CF33
:1000100006F00001E9CF0CF0EACF07F0E1CF08F0DD
:10002000E2CF09F0D9CF0AF0DACF0BF0F3CF12F01C
:10003000F4CF13F0FACF14F0F5CF15F0F6CF16F099
:10004000F7CF17F000C00EF001C00FF002C010F0A3
:1000500003C011F0F2AA30EF00F0F2B4A2EF01F009
:100060009DA036EF00F09EB0ACEF01F09DAA3CEFF2
:1000700000F09EBA09EF02F09DA842EF00F09EB892
:100080008AEF02F00EC000F00FC001F010C002F0C5
:1000900011C003F00CC0E9FF07C0EAFF078E08C0DB
:1000A000E1FF09C0E2FF0AC0D9FF0BC0DAFF12C0AE
:1000B000F3FF13C0F4FF14C0FAFF15C0F5FF16C01C
:1000C000F6FF17C0F7FF045006C0E0FF05C0D8FFD9
:1000D0001000E00FF66E000EF7220900F550120036
:1000E000FF0366034C03320319030003E702CF0248
:1000F000B702A0028A0274025F024A02360222029A
:100100000F02FD01EB01DA01C901B901A9019A0150
:100110008B017D016F016201550149013D013201F1
:1001200028011E0114010A010101F700EF00E60099
:10013000DE00D600CE00C700C000B900B300AC009E
:10014000A600A1009B00960090008C008700820012
:100150007E007A00760072006E006A00670063001D
:1001600060005D005A005700540052004F004D00DF
:100170004A00480046004400420040003E003C0067
:100180003A003800370035003300320030002F00CD
:100190002E002C002B002A00290027002600250015
:1001A000240023002200210020001F001E001D004B
:1001B0001C001B001B001A00190018001700170074
:1001C0001600150015001400130013001200110092
:1001D0001100100010000F000E000E000D000D00A9
:1001E0000C000C000000F76AF60FF66E010EF72205
:1001F0000900F55012003437313037300000F76A0B
:100200000E0FF66E020EF7220900F5501200303084
:10021000303330370000F76A260FF66E020EF722F1
:100220000900F55012003030303131310000F76AEA
:100230003E0FF66E020EF7220900F5501200303024
:10024000303131320000F76A560FF66E020EF72297
:100250000900F55012003030303434300000F76AB5
:100260006E0FF66E020EF7220900F55012003030C4
:10027000303434310000F76A860FF66E020EF72232
:100280000900F55012003030303434320000F76A83
:100290009E0FF66E020EF7220900F5501200303064
:1002A00030343433000073746174653A5B4F4E5DD3
:1002B000000073746174653A5B4F46465D00457893
:1002C000697400004368616E676520686F7365003C
:1002D000496E697420706973742E20706F7300000A
:1002E0004D6F766520706973746F6E002120496EC2
:1002F0006974207265656C20210020202020000098
:10030000202020200000206F6B20000020202020D3
:10031000000020202B200000206F6E200000206FA6
:100320006B20000020202020000020202D20000035
:10033000206F666600005365742070617373776F79
:1003400072640000D59EAB888194F29442EF00F075
:100350009EA8FED7AD6E1200F70ECF6ECE6A0400D7
:10036000222A22500A0801E1226A4B5201E04B0680
:10037000225228E14B5226E10101996B9951030861
:1003800018E3036A99514D0FE96E000E0320EA6EDF
:10039000EF520DE0036A99514D0FE96E000E0320F4
:1003A000EA6EEF6A9951100DF3CF24F002D0992B29
:1003B000E5D7040E426E256AAB988184010E0001D8
:1003C000C7DF9D88225005080AE14B5208E1070E5D
:1003D000426E256AAB988184010EBADF9D882C2A73
:1003E0002C50140802E12C6A1C882B2A2B5064081C
:1003F00002E12B6A1C869E9042EF00F09EAAFED777
:10040000ABCF1BF0AECF01F01BA202D0AB98AB88F4
:1004100012004250040833E1036A3C50340FE96E85
:10042000000E0320EA6EEACF9CF1E9CF9BF1E6DFF4
:100430009CC1EAFF9BC1E9FF01C0EFFF3C2A3C5091
:1004400008081CE13C6A3C5006080BE3036A3C5078
:10045000340FE96E000E0320EA6EEF503E263C2A70
:10046000F2D73B503E5C0AE134C026F026500F0B19
:10047000516E35C088F036C087F01D8648D0425096
:1004800007083CE1036A4350440FE96E000E032065
:10049000EA6EEACF9CF1E9CF9BF1B0DF9CC1EAFFA5
:1004A0009BC1E9FF01C0EFFF432A4350060825E145
:1004B000436A435004080BE3036A4350440FE96E58
:1004C000000E0320EA6EEF503E26432AF2D7495031
:1004D0003E5C13E144C08CF045C08BF0030E5A6EB5
:1004E000462C0AD04A2A4A50020805E2320E4B6EC8
:1004F000426A4A6A576A01D04A6A09D07FDF01C05E
:1005000043F04B5204E0432C02D0320E4B6E9E9AC5
:1005100042EF00F0425004084FE1255007E0010A85
:1005200014E0030A1BE0010A29E044D0315202E141
:10053000000E01D0010E800DF350040F0101996FE0
:100540009951000105DF252A36D0030E242401012C
:10055000996F99510001FCDE252A2DD02450242AC0
:10056000036A230FE96E010E0320EA6EEFCF99F1C3
:10057000010199510001ECDE252A1DD024500F0BFA
:100580000FE02450242A036A230FE96E010E032092
:10059000EA6EEFCF99F1010199510001D9DE09D03E
:1005A0009D98020ED5DE3F0E24163C6A436A3E6AD1
:1005B000D58E01D0246A2FD0425007082CE1255057
:1005C00005E0010A0EE0030A1FE025D05750200D78
:1005D000F350070F0101996F99510001B9DE252AE7
:1005E0001AD0000E1DBC010E030F0101996F995125
:1005F0000001AEDE252A1DAC06D04C2A4C50020864
:1006000002E24C6A1D9C07D09D98020EA1DE3C6A56
:10061000436A3E6AD58E9E9842EF00F04D6F726538
:1006200020696E666F2E0000262066756E63746901
:100630006F6E730074656D702031000074656D70AD
:10064000203200004A70313A20004A70323A2000CD
:100650005661633A2000436F6E74726F6C005345AD
:1006600050323400526573657420636F756E746523
:1006700072202020000032335F32354B32325F313E
:100680002E342E63000032312D4E6F762D32310024
:1006900031393A33393A353700005265626F6F7439
:1006A0000000534550323300496E7465726C6F63BD
:1006B0006B00696E616374697661746564005B20C8
:1006C000256C75205D2073742E006D6561737572E5
:1006D00065642074656D702E00002077617465720A
:1006E0003A00736C756467653A00696E707574736F
:1006F0002026206F7574707574730000416E616CF4
:100700006F67206F75742E0076616C75653A000016
:100710002573203137007465726D00006C6F77654A
:1007200072206C69676874006F75742E322074656E
:10073000726D2E20313800007570706572206C6902
:10074000676874006F75742E33207465726D2E2087
:100750003139000076616C7665006F75742E362035
:100760007465726D2E20323200006C6174636820F3
:1007700073776974636800006F75742E3720746531
:10078000726D2E203233000076616370756D7000DB
:100790006F75742E35207465726D2E203231000015
:1007A0006F7074696F6E0000696E2E31207465720F
:1007B0006D2E20330000626C6F7765722070756D4E
:1007C0007000696E2E34207465726D2E2036000024
:1007D0006C61746368207377697463680000696E84
:1007E0002E35207465726D2E203135006A65747067
:1007F000756D7000696E2E36207465726D2E203115
:10080000360076616C75652E0000616E61696E2E32
:1008100031207465726D2E20370076616C75652EFF
:100820000000616E61696E2E32207465726D2E203B
:1008300038006F7074696F6E2000616E61696E2E92
:1008400033207465726D2E20390074656D7020310F
:100850000000616E61696E2E34207465726D2E2009
:100860003130000074656D7020320000616E616986
:100870006E2E35207465726D2E2031310000617549
:10088000746F6D61746963006C696E656172697A19
:100890006174696F6E005374617475733A5B4F4B8A
:1008A0005D005374617475733A5B6E4F4B5D00006D
:1008B0006C696E6561722E64617461002573253206
:1008C000752225356C752273656B00007469643A76
:1008D00000006C69743A00006F7074696F6E0000FC
:1008E000696E2E32207465726D2E203400006F7098
:1008F00074696F6E0000696E2E33207465726D2E00
:10090000203500006D616EF67665722070726F7032
:1009100000006F75742E34207465726D2E20323095
:1009200000006F7074696F6E00006F75742E382050
:100930007465726D2E203234000073657474696EB4
:10094000677300007365742072706D0072706D3A89
:1009500025356C75000063616C2E766F6C2E7365A7
:100960006E7300007265663A25336C752067697690
:100970003A25346C75004F4B20746F207361766597
:1009800020202020202000006F6C64207265663AD1
:1009900020202020000063616C2E7072652E73652C
:1009A0006E7300007265663A253375206769763A82
:1009B00025346C7500004F4B20746F207361766591
:1009C00020202020202000006F6C64207265663A91
:1009D0002020202000006D61782E20766F6C756DD0
:1009E000650076616C75653A000054656D706C69E0
:1009F0006D69740076616C75653A0000214C6F7703
:100A0000206C6576656C00006C697465723A000054
:100A100072616D70696E670076616C75653A000091
:100A2000616E616C6F672063656E746572007661DC
:100A30006C75653A0000616E612E206F75742072CE
:100A400065642E31000076616C75653A000074654E
:100A5000726D0000616E612E206F75742072656486
:100A60002E32000076616C75653A00007465726D17
:100A70000000616E612E206D6178000076616C75FA
:100A8000653A0000616E612E207072696F2031003E
:100A900076616C75653A00007465726D000064657E
:100AA0006C6179206A657470756D700025327520EF
:100AB0007820323030206D5300007020666F722035
:100AC000636C6F73650076616C75653A000045452F
:100AD0002061646472657373000045453A00766175
:100AE0006C75650070617373776F726400003233E8
:100AF0005F32354B32325F312E342E63000032319B
:100B00002D4E6F762D32310031393A33393A35373F
:100B1000000070617373776F7264206661696C6541
:100B20006400686967682074656D7000776174653A
:100B3000720063757272656E740074656D706572B3
:100B4000617475723A00257325356C752062617287
:100B500000005061696E653A2000257325356C757B
:100B60002070736900005061696E653A200025733A
:100B700025356C75206C697400004DE4E472E43A2C
:100B80002000257325356C752067616C00004DE4ED
:100B9000E472E43A20004DE4E472E43A2021566520
:100BA00073692076E46800002D2D4C6973E4E4201D
:100BB00076657474E4212D2D0000257325356C7540
:100BC0002072706D00004D6F6F74743A20004B6599
:100BD0006C61203A2000206D657400002573256348
:100BE00025336C752E25316C75206D6574004C6550
:100BF000746B753A00002A204C65746B75206F6821
:100C00006A61696E202A0000257325336C75207394
:100C1000656B3A25356C750041643A006164723A3F
:100C2000000074696D652076616C756500006C6FFD
:100C30006767656420696E20454570726F6D0000BE
:100C4000010EEA6E750EE96EEF500EE0020E016EB7
:100C5000006A002EFED7012EFBD7620E006E002E1A
:100C6000FED700D0EF2EF2D712000101866BF2CF33
:100C700087F1F29E81C1A9FFA69CA69EA680A850DE
:100C800087BFF28E856F822D17D0812BF2CF87F12F
:100C9000F29E81C1A9FFA69CA69EA680A85087BFF0
:100CA000F28E866F86C184F185C183F183C101F024
:100CB00084C102F008D003D0846B85C183F183C165
:100CC00001F084C102F00001120001017F6B7BC1C1
:100CD0007EF1F250006EF29E7AC1A9FF7EC1A8FF9C
:100CE000A69CA69EA6840F01550EA76EAA0EA76EFF
:100CF000A682A6B2FED7A6940050F21201017D2D65
:100D000019D07CC17FF17A2BF250006EF29E7AC12D
:100D1000A9FF7FC1A8FFA69CA69EA6840F01550E21
:100D2000A76EAA0EA76EA682A6B2FED7A694005002
:100D3000F21201011E840001120001017B517D03AA
:100D4000F3CF01F0F4CF00F07E03F35000267C5186
:100D50007D03F3500020026E00011200016A026A56
:100D6000006A036A01017F5102E17E5118E0100E12
:100D7000806FD8907C377D37003603367F51035C17
:100D800002E17E51005C07E37E51005ED8A00306BD
:100D90007F51035ED88001360236802FEAD70001EA
:100DA000120074C1C2FF120E006E002EFED7C28266
:100DB000C2B2FED7050E006E002EFED700D0010194
:100DC0007C6BC4CF7BF1010E7E6F7D6B0001B5DFC4
:100DD000C35001010124786F000E0220796F745115
:100DE000030A000109E0040A20E00C0A43E0040AB7
:100DF00042E01C0A41E040D0FC510101795D0FE363
:100E000005E10001FB510101785D09E30001FB519F
:100E10000101785F0001FC510101795B04D0000EF3
:100E2000016E026E7DD0000127D079C17CF178C1BE
:100E30007BF101017E6B0A0E7D6F00017EDF02C037
:100E40007BF101C07AF102C07DF101C07CF10101AA
:100E50007F6B210E7E6F000181DF02C07BF101C03C
:100E60007AF132500101015C786F000E0258796FFF
:100E7000000102D001D000D0010177534DE076513E
:100E8000795D22E303E17851755D1EE27551785D6D
:100E90007A6F765179597B6F7D6F7AC17CF17F6B68
:100EA0000A0E7E6F00015ADF02C07BF101C07AF1A9
:100EB000010E01010124016E000E0220036E01509B
:100EC00075270350762322D07951765D1FE303E125
:100ED0007551785D1BE27851755D7A6F795176595D
:100EE0007B6F7D6F7AC17CF17F6B0A0E7E6F000194
:100EF00035DF01C07AF1010E01010124016E000EFF
:100F00000220036E0150755F0350765B75C101F0DE
:100F10007651026E05D004D078C101F079C102F09B
:100F2000000112000101746B74513F080BE3036A66
:100F30007451230FE96E010E0320EA6E200EEF6E4E
:100F4000742BF2D7746B745103080BE3036A74516A
:100F50004D0FE96E000E0320EA6E010EEF6E742B4A
:100F6000F2D7236A000112000101926B936B010E0C
:100F7000946FDA6AD96A976F8A0E966F010EEA6EDD
:100F80008E0EE96E97C1E2FF96C1E1FF94C195F123
:100F9000D890E550EE02F3509223F4509323952F0E
:100FA000F7D792C1DEFF93C192F1936BD8B0932B28
:100FB000962BD8B4972B942B94510508DFE10001B0
:100FC0001200D8B204D0010EEA6E940EE96E006AE7
:100FD000016A026A036A0101946B956B966B976BC9
:100FE00093519211911190112CE0200E986FD8908E
:100FF0008C378D378E378F379437953796379737AD
:101000009351975D08E19251965D05E19151955D8F
:1010100002E19051945D0FE39051945F9151D8A0FB
:10102000913D955F9251D8A0923D965F9351D8A083
:10103000933D975FD8800036013602360336982FED
:10104000D6D794C1EFFF95C1ECFF96C1ECFF97C1D5
:10105000ECFF00011200010182C08BF181C08AF116
:101060008D6B8C6B916B906B030E8F6FE80E8E6F98
:1010700000017ADF03C077F102C076F101C075F19B
:1010800000C074F10F0E0101816F010E826F00012B
:10109000ECDD01017F6B7E6B02C07DF101C07CF154
:1010A000306A3050285CD8A07ED0D8903034800F81
:1010B000806F816F010E826F0001D7DD01017B6BB4
:1010C0007A6B02C079F101C078F1D8903034036AAC
:1010D0008F0FE96E000E0320EA6EEACF83F1E9CFAD
:1010E00082F1D89277C18FF176C18EF175C18DF101
:1010F00074C18CF17FC193F17EC192F17DC191F1F8
:101100007CC190F100015DDF83C1EAFF82C1E9FF8C
:1011100003C087F102C086F101C085F100C084F1EF
:10112000EACF89F1E9CF88F103C08DF102C08CF1DB
:1011300001C08BF100C08AF17BC191F17AC190F1BD
:1011400079C18FF178C18EF10FDF89C1EAFF88C1C3
:10115000E9FF03C087F102C086F101C085F100C03C
:1011600084F1EACF8BF1E9CF8AF1D89203C08FF1F5
:1011700002C08EF101C08DF100C08CF10101936BB2
:10118000926B030E916FE80E906F00011ADF8BC116
:10119000EAFF8AC1E9FF01C0ECFFED5200C0EFFF9A
:1011A000302A01017ED700012DEF12F001017751A5
:1011B000100DF3507825236E3F0E23160001120008
:1011C00001017F5324E0036A2350230FE96E010ECF
:1011D0000320EA6E7F51EF5C16E0036A2350230F71
:1011E000E96E010E0320EA6E7FC1EFFF2338006E27
:1011F0000F0E00160050036A4D0FE96E000E03201B
:10120000EA6E010EEF6E23503E0801E3232A00012F
:1012100012000900F5520CE0F6CF77F1F7CF78F124
:10122000F5CF7FF1CDDF77C1F6FF78C1F7FFF1D7BA
:101230001200036A2350230FE96E010E0320EA6EA9
:10124000EF50200816E0036A2350230FE96E010EC9
:101250000320EA6E200EEF6E2338006E0F0E00168C
:101260000050036A4D0FE96E000E0320EA6E010E76
:10127000EF6E232A23500F0BDCE11200006A016A93
:1012800001017751D89078B100260032013278B34D
:1012900000260032013278B500260032013278B7DC
:1012A00000260032013278B900260032013278BBC4
:1012B00000260032013278BD00260032013278BFAC
:1012C00000260032013200011200030E0101776F87
:1012D000786B00016BDF0101776B7551F00B786F54
:1012E00077530AE1785308E1FA0EF66E020EF76EB4
:1012F00000018FDF1DD00101776B7551F00B786F06
:10130000775317E17851100814E1200E7F6F000128
:1013100057DF7F0E01017F6F000152DF200E0101B8
:101320007F6F00014DDF200E01017F6F000148DF5C
:101330000101776B75510F0B786F77530AE1785382
:1013400008E1000EF66E030EF76E000162DF2DD08D
:101350000101776B75510F0B786F775317E1782D7B
:1013600015D0200E7F6F00012BDF7E0E01017F6FF5
:10137000000126DF200E01017F6F000121DF200E1A
:1013800001017F6F00011CDF10D00101776B7551E7
:101390000F0B786F77530AE17851040807E1060EC6
:1013A000F66E030EF76E000134DF01017451F00B8D
:1013B000776F786B77530AE1785308E10C0EF66E7D
:1013C000030EF76E000125DF50D001017451F00BC0
:1013D000776F786B7751100817E1785315E1200E7D
:1013E0007F6F0001EDDE200E01017F6F0001E8DE5E
:1013F000060E01017F6F0001E3DE200E01017F6F09
:101400000001DEDE32D001017451F00B776F786B92
:10141000775120080AE1785308E1120EF66E030EA8
:10142000F76E0001F6DE21D001017451F00B776FE9
:10143000786B775130080AE1785308E1180EF66EA0
:10144000030EF76E0001E5DE10D001017451F00BC0
:10145000776F786B7751400809E1785307E11E0EEA
:10146000F66E030EF76E0001D4DE010174510F0B0E
:10147000776F786B77530AE1785308E1240EF66EA4
:10148000030EF76E0001C5DE3ED0010174510F0B53
:10149000776F786B772D17D0785315E1200E7F6F1B
:1014A00000018EDE200E01017F6F000189DE050E36
:1014B00001017F6F000184DE200E01017F6F0001BA
:1014C0007FDE21D0010174510F0B776F786B77515C
:1014D00002080AE1785308E12A0EF66E030EF76E51
:1014E000000197DE10D0010174510F0B776F786BFC
:1014F0007751030809E1785307E1300EF66E030EC9
:10150000F76E000186DE01011DAE06D0515203E1E7
:101510001D9E026B016B3DD15152D8B41FD11EB636
:1015200004D0006B0001FF6B0101765304E11D8EB6
:10153000010E526E2AD002C178F10151012BD8B4AC
:10154000022B776F775305E1785303E1010E526E5A
:101550001CD0025303E10151280806E2765102082B
:1015600003E1140E526E11D0025303E1015114082D
:1015700003E2050E526E09D0025303E10151070840
:1015800003E2010E526E01D0526A776B7551F00B77
:10159000786F775311E1785110080EE15150080827
:1015A0000BE10001FD51D8B4FE07FD071D8E000EB2
:1015B000016EF2D0D1D00101776B75510F0B786FAE
:1015C00077530FE1782D0DD0515004080AE1000146
:1015D000FD2BD8B4FE2B1D8E000E016EDDD0BCD0CD
:1015E0000101776B75510F0B786F775310E17851CC
:1015F00004080DE1515004080AE10001FD2BD8B4A4
:10160000FE2B1D8E000E016EC7D0A6D001017451B5
:10161000F00B776F786B775110081EE178531CE15F
:101620005150020819E10001FD5188080CE1FE51FA
:10163000130809E152C077F10101786900011EDE4B
:101640000150AAD007D0E80EFD5F030EFE5B000E2E
:10165000016EA2D081D0010174510F0B776F786BAE
:10166000772D18D0785316E1512C14D00001FD517C
:10167000880807E1FE51130804E152C001F08CD044
:1016800007D0E80EFD27030EFE23000E016E84D066
:1016900063D001017451F00B776F786B775120089C
:1016A0000BE1785309E15150020806E152C001F004
:1016B000000172D051D0010174510F0B776F786B1C
:1016C000775102080DE178530BE1512C09D052C03B
:1016D00077F178690001D2DD01505ED03DD0010183
:1016E0007451F00B776F786B775130080BE17853BA
:1016F00009E15150020806E152C001F000014CD04E
:101700002BD0010174510F0B776F786B7751030861
:101710000DE178530BE1512C09D052C077F1786973
:101720000001ACDD015038D017D001017451F00B2D
:10173000776F786B775140080BE1785309E151508E
:10174000020806E152C001F0000126D005D00101D7
:10175000000E016E000120D01BD00101026B016B55
:101760001EB017D000C103F00001FF51FF2BD8A419
:1017700002D00101002B0101776F03C078F178538B
:1017800003E17751C80805E20001FE6BFD6B1E9670
:101790000101000E016E0001120001017B51016A7E
:1017A0007A5D03E27AC100F00CD0006A080E7C6F0B
:1017B0007A3700367B51005CD8B0006E01367C2F42
:1017C000F7D700011200200E010175A9300E766FC7
:1017D00074C100F000AE08D0001E002A00C074F1F1
:1017E0002D0E766F758F7581015074C17AF1640E7C
:1017F0007B6F0001D2DF00C074F1300E01240101C3
:10180000776F74C17AF10A0E7B6F0001C6DF300E6C
:1018100000240101796F300E0124786F76C100F049
:10182000300E775D04E0758375BF758512D076C183
:1018300077F1200E766F300E785D04E0758175BF0C
:10184000758307D0D8A4758104E177C178F1200EA3
:10185000776F75B505D075B307D075B109D00CD0C9
:1018600076C17FF10001ACDC77C17FF10001A8DC1B
:1018700078C17FF10001A4DC79C17FF10001A0DC17
:10188000120074C181F1010E0101826F000135EC7B
:1018900006F002C06AF001C069F0020E0101742571
:1018A000776F816F826B000135EC06F001C029F083
:1018B000030E01017425776F816F826B000135EC97
:1018C00006F001C02AF01CB004D01CB202D01CA447
:1018D000CAD00101765306E175510F08D8A002D095
:1018E0000001C1D076C17DF175C17CF10E0E7F6F14
:1018F000100E7E6F0001AEEC06F001506927025019
:101900006A2376C17DF175C17CF10E0E01017F6FF6
:10191000100E7E6F0001AEEC06F000C077F1010101
:1019200003C078F103C07DF100C07CF17F6B3C0EF9
:101930007E6F0001AEEC06F00150292676C17DF1E4
:1019400075C17CF10E0E01017F6F100E7E6F0001DC
:10195000AEEC06F000C077F1010103C078F176C16A
:101960007DF175C17CF10E0E7F6F100E7E6F000150
:10197000AEEC06F000C079F1010103C07AF103C0BA
:101980007DF100C07CF17F6B3C0E7E6F0001AEEC00
:1019900006F002C07AF101C079F102C07CF101C009
:1019A0007BF101017E6B3C0E7D6F00019DEC06F02A
:1019B00001500101775D006E0250785900502A26CF
:1019C0002A503B0812E22AC07AF13C0E7B6F0001DC
:1019D000E4DE015029262AC07AF13C0E01017B6F1A
:1019E0000001DBDE00C02AF0010129503B0814E2AF
:1019F00029C07AF13C0E7B6F0001CFDE01506927D0
:101A0000000E6A2329C07AF13C0E01017B6F0001B0
:101A1000C4DE00C029F0010174C17AF16AC07CF112
:101A200069C07BF1010E7D6F000165EC06F0020ECE
:101A300001017425776F796B786F7A6F7C6B29C0A1
:101A40007BF17D6B000165EC06F0030E010174254E
:101A5000776F796B786F7A6F7C6B2AC07BF17D6BC7
:101A6000000165EC06F01200EACF7EF1E9CF7DF1CE
:101A700001017739F009796F7927E20F7A6F320F18
:101A80007C6F77510F0B7A277A277C27E90F7B6FC2
:101A90007B277B2776390F0B7B277C277B377C378F
:101AA0007C1F7C3776510F0B7C277937070E786FB8
:101AB0000A0E7B077C27FDE37A077B27FDE3790786
:101AC0007A27FDE378077927FDE3010EEA6E780EA9
:101AD000E96E070E7D157D9DE926000EEA22E9508C
:101AE0007C0803E1EA2C01D07D8DEF50006E08E107
:101AF0007DBD06D07DB916D07DB702D0200E03D0B3
:101B00007D877D99300E0026EACF77F1E9CF76F117
:101B100000C07FF10001E0EC08F077C1EAFF76C178
:101B2000E9FF0101EE507DADDAD70001120001504E
:101B300076C17AF1640E01017B6F00012EDE00C0D8
:101B400076F10150300E08E1010177A310D077B78C
:101B50000ED077B9200E04D001017797779977815D
:101B6000012601C07FF10001E0EC08F0010176C11F
:101B70007AF10A0E7B6F000110DE00C076F1015091
:101B8000300E08E1010177B70BD077A109D077B902
:101B9000200E0001012601C07FF1E0EC08F00101F8
:101BA000300E762776C17FF10001E0EC08F01200DC
:101BB0000900F6CF77F1F7CF78F1F5CF7FF1E0ECC0
:101BC00008F077C1F6FF78C1F7FF0101762F01D049
:101BD00002D00001EDD7000112000101759174518E
:101BE000010A00011BE0030A1FE0010A23E0070AC3
:101BF00027E0010A2BE0030A2FE0010A33E00F0A75
:101C000037E0010A3BE0030A3FE0010A43E0070A2C
:101C100047E0010A4BE0030A4FE054D082A203D010
:101C20000101758100014ED081A603D001017581AB
:101C3000000148D082A003D001017581000142D08B
:101C400082AA03D00101758100013CD082A803D093
:101C500001017581000136D082A403D00101758194
:101C6000000130D082A603D00101758100012AD085
:101C700080A803D001017581000124D081BE03D06A
:101C80000101758100011ED081BC03D00101758165
:101C9000000118D081BA03D001017581000112D072
:101CA00081B803D00101758100010CD081B203D04D
:101CB00001017581000106D081B003D00101758159
:101CC000000100D0010175A109D0A60EF66E020E2A
:101CD000F76E000109EC09F008D00101B20EF66EB2
:101CE000020EF76E000109EC09F012000101776B9A
:101CF000786B0001D6EC08F0360EF66E030EF76E28
:101D000009EC09F019EC09F0010E0101776F786B0D
:101D10000001D6EC08F0010E546E545006080DE395
:101D2000036A5450640FE96E010E0320EA6EEFCF90
:101D30007FF1E0EC08F0542AF0D719EC09F0020E1C
:101D40000101776F786B0001D6EC08F0010E546E3C
:101D5000545006081AE3A00EFD5D006E0F0EFE59EA
:101D6000036E0050545C09E1035207E12D0E01019E
:101D70007F6F0001E0EC08F006D0200E01017F6FBC
:101D80000001E0EC08F0542AE3D719EC09F0120046
:101D90000101785302E179533EE075C1EAFF74C155
:101DA000E9FFEFCF7AF177C1EAFF76C1E9FFEF50A3
:101DB0007A5D17E075C103F074C1E9FF03C0EAFF63
:101DC000EFCF7AF177C103F076C1E9FF03C0EAFFF4
:101DD000EF507A5D02E2FF0E01D0010E016E1DD0C0
:101DE00009D075C1EAFF74C1E9FFEF5203E1000EAB
:101DF000016E13D075C103F07451742BD8B4752BD8
:101E000077C103F07651762BD8B4772B7851D8B4BC
:101E100079077807BED7000E016E0001120001019C
:101E20007551000A000109E0010A0EE0030A13E0FF
:101E3000010A18E0070A1DE023D0BE0EF66E020E5E
:101E4000F76E09EC09F01CD0C40EF66E020EF76EA8
:101E500009EC09F015D0D00EF66E020EF76E09EC03
:101E600009F00ED0E00EF66E020EF76E09EC09F0E6
:101E700007D0EC0EF66E020EF76E09EC09F000D0FA
:101E8000120001017F518119800B836F7FAF05D054
:101E90007E1F7F1F7E2BD8B47F2B81AF05D0801F84
:101EA000811F802BD8B4812B7E518003F3CF01F0AA
:101EB000F4CF00F08103F35000267F518003F350EC
:101EC0000020026E83AF05D0011E021E012AD8B485
:101ED000022A0001120001017B91140E76257D6F0C
:101EE0007F6B7E6F7EBF7F07816B020E806F00016C
:101EF000C8DF02C003F0015002C0F7FF69EC00F038
:101F00000900F5CF03F00101776F03C078F1150EDA
:101F100076257D6F7F6B7E6F7EBF7F07816B020EA4
:101F2000806F0001AEDF02C003F0015002C0F7FF76
:101F300069EC00F00900F5CF03F00101796F03C0EF
:101F40007AF175517A5D06E303E17951745D02E23D
:101F5000762B0AD07851755D06E303E17451775D05
:101F600002E2760701D07B817BA1B7D776C101F071
:101F7000000112000A0E0101756F000120EC06F04D
:101F800081A00DD01CA00BD00101746B7CC076F138
:101F90007BC075F1000175DC1C9038D008D081B091
:101FA00006D01CB004D01C807C6B7B6B2FD01DA096
:101FB0000ED01CA20CD0040E0101746F7EC076F10D
:101FC0007DC075F100015DDC1C9220D008D01DB0F1
:101FD00006D01CB204D01C827E6B7D6B17D081A80A
:101FE0000ED01CA40CD0080E0101746F80C076F1D5
:101FF0007FC075F1000145DC1C9408D007D081B882
:1020000005D01CB403D01C84806B7F6BBDEF2DF01A
:10201000010175517719800B796F75AF05D0741F69
:10202000751F742BD8B4752B77AF05D0761F771F2B
:10203000762BD8B4772B016A026A006A036A77515B
:1020400002E1765118E0100E786FD890743775372A
:10205000003603367751035C02E17651005C07E3FA
:102060007651005ED8A003067751035ED880013612
:102070000236782FEAD779AF05D0011E021E012A59
:10208000D8B4022A00011200F86AD09E078EFE0E14
:10209000006E060E016E020EE96E000EEA6EEE6A2A
:1020A0000400002EFCD7012EFAD71B6AB896050E45
:1020B000AF6EA20EAC6E900EAB6E0101736B726BC5
:1020C0000F01386B396B3A6B776A786A796A196AEB
:1020D0001A6A2F0E926EF30E936E800E946E896ABA
:1020E0008A6A8B6A280E0101756F000120EC06F0E8
:1020F000609060926094810EC06E0A0EC16E1D8069
:102100001E881E9EB40E316E1D82D1804F0E0101BD
:10211000816F826B000135EC06F001C000F00250C7
:10212000036E02E1005210E0035003E1010E005C77
:102130000EE0035003E1020E005C0CE0035003E1EB
:10214000030E005C0AE00BD01F901F9208D01F8086
:102150001F9205D01F801F8202D01F901F820C0E7D
:102160000101816F010E826F000135EC06F002C0A3
:1021700082F001C081F00E0E0101816F826B0001BF
:1021800035EC06F001C028F0600E0101816F010EF0
:10219000826F000135EC06F002C0FCF001C0FBF0DC
:1021A000460E0101816F826B000135EC06F001C023
:1021B00032F0480E0101816F826B000135EC06F0B0
:1021C00001C033F04E0E0101816F826B000135ECCE
:1021D00006F001C05BF05B5202E1010E5B6E410E46
:1021E0000101816F826B000135EC06F001C02EF019
:1021F0002E5202E01C8A01D01C9A420E0101816F0E
:10220000826B000135EC06F001C02FF0490E010190
:10221000816F826B000135EC06F001C061F0700E39
:102220000101816F826B000135EC06F01D9A01B04F
:102230001D8A5F0E0101816F826B000135EC06F093
:1022400002C0FAF001C0F9F0620E0101816F010EC7
:10225000826F000135EC06F002C00EF101C00DF1F5
:102260001D0E0101816F826B000135EC06F001C08B
:1022700063F0220E0101816F826B000135EC06F0E4
:1022800001C064F01B0E0101816F010E826F00011D
:1022900035EC06F002C084F001C083F01DAA0FD017
:1022A000832BD8B4842B1B0E01017A6F84C07CF180
:1022B00083C07BF1010E7D6F000165EC06F0270EF7
:1022C0000101816F010E826F000135EC06F002C042
:1022D00014F101C013F101011351141101E01E8228
:1022E000290E816F010E826F000135EC06F002C0ED
:1022F00016F101C015F12B0E0101816F010E826FE5
:10230000000135EC06F002C018F101C017F12D0EE6
:102310000101816F010E826F000135EC06F002C0F1
:102320001AF101C019F12F0E0101816F010E826FA8
:10233000000135EC06F002C01CF101C01BF1320EA9
:102340000101816F010E826F000135EC06F002C0C1
:1023500020F101C01FF1310E0101816F826B00017C
:1023600035EC06F001C05CF05C5202E1010E5C6EDF
:10237000C150F00BC16E2F0E0F01386F000E396F78
:102380003A6F030E0101746F6CC076F16BC075F18A
:10239000776B0001D1EC06F002C06CF001C06BF06D
:1023A000070E0101746F6EC076F16DC075F1776B29
:1023B0000001D1EC06F002C06EF001C06DF00F0E0E
:1023C0000101746F72C076F171C075F1776B000115
:1023D000D1EC06F002C072F001C071F0130E0101E1
:1023E000746F74C076F173C075F1776B0001D1EC36
:1023F00006F002C074F001C073F00B0E0101746F9F
:1024000070C076F16FC075F1776B0001D1EC06F00A
:1024100002C070F001C06FF0370ECD6ECC6AC20EF4
:10242000D56E1EA211D08B920C0E666E656A646A20
:10243000010E636EE70E0F014917000E49130409E0
:10244000BA6EFF0EBB6E00019D80F28A9D8AC00E9F
:10245000F21292EC07F02BEF08F0C80E0101756F35
:10246000000120EC06F01EA213D014C102F013C12B
:1024700001F00232013202320132023201C067FF42
:1024800002320230300B006E6650CF0B0010666EC9
:1024900014C11EF113C11DF1216A0101046B010E6B
:1024A000036F90C076F08FC075F0030E5A6E000176
:1024B000FD51FE11D8B4CCEF2AF01DA6CCEF2AF0C6
:1024C0001D96515009080AE1216AFE6BFD6B1E96AC
:1024D0000101006BC80E0001FF6F536A51500F08D5
:1024E0000DE1030EFE6FE80EFD6F1D8E0101006B06
:1024F000A00E0001FF6F536A1E96576A51500C08D8
:102500000CE1130EFE6F880EFD6F1D8E0101006B36
:102510000001FF6B576A586A566AFDC000F0FEC0A2
:1025200003F0030EFE5D04E1E80E005CD8B4C6D1F2
:10253000030E035C04E1E90E005CD8B4F0D1030E95
:10254000035C04E1EA0E005CD8B456D2030E035CCF
:1025500004E1EB0E005CD8B424D3030E035C04E169
:10256000EC0E005CD8B455D3030E035C05E1ED0E10
:10257000005CD8B44AEF16F0030E035C05E1EE0EE2
:10258000005CD8B496EF16F0030E035C05E1EF0E85
:10259000005CD8B4CCEF16F0030E035C05E1F00E3E
:1025A000005CD8B425EF17F0070E035C05E1D00EF0
:1025B000005CD8B483EF17F0070E035C05E1D10E81
:1025C000005CD8B4ADEF17F0070E035C05E1D20E46
:1025D000005CD8B4FBEF17F0070E035C05E1D30EE7
:1025E000005CD8B43EEF18F0070E035C05E1D40E92
:1025F000005CD8B481EF18F0070E035C05E1D50E3E
:10260000005CD8B4C4EF18F0070E035C05E1D60EE9
:10261000005CD8B407EF19F0070E035C05E1D70E94
:10262000005CD8B44AEF19F0070E035C05E1D80E40
:10263000005CD8B480EF19F0070E035C05E1D90EF9
:10264000005CD8B4B6EF19F0070E035C05E1DA0EB2
:10265000005CD8B4ECEF19F0070E035C05E1DB0E6B
:10266000005CD8B422EF1AF0070E035C05E1DC0E23
:10267000005CD8B469EF1AF0070E035C05E1DD0ECB
:10268000005CD8B4B0EF1AF0070E035C05E1DE0E73
:10269000005CD8B4F7EF1AF0070E035C05E1DF0E1B
:1026A000005CD8B43EEF1BF0070E035C05E1E00EC2
:1026B000005CD8B485EF1BF0070E035C05E1E10E6A
:1026C000005CD8B4F9EF1BF0070E035C05E1E20EE5
:1026D000005CD8B4A2EF1CF0070E035C05E1E30E2A
:1026E000005CD8B4D8EF1CF0070E035C05E1E40EE3
:1026F000005CD8B40EEF1DF0070E035C05E1E50E9B
:10270000005CD8B451EF1DF00B0E035C05E1B80E70
:10271000005CD8B494EF1DF00B0E035C05E1B90E1C
:10272000005CD8B4BFEF1DF00B0E035C05E1BA0EE0
:10273000005CD8B470EF1EF00B0E035C05E1BB0E1D
:10274000005CD8B443EF1FF00B0E035C05E1BC0E38
:10275000005CD8B40DEF20F00B0E035C05E1BD0E5C
:10276000005CD8B497EF20F00B0E035C05E1BE0EC1
:10277000005CD8B417EF21F00B0E035C05E1BF0E2F
:10278000005CD8B4A9EF21F00B0E035C05E1C00E8C
:10279000005CD8B435EF22F00B0E035C05E1C10EEE
:1027A000005CD8B4BCEF22F00B0E035C05E1C20E56
:1027B000005CD8B455EF23F00B0E035C05E1C30EAB
:1027C000005CD8B4EEEF23F00B0E035C05E1C40E01
:1027D000005CD8B475EF24F00B0E035C05E1C50E68
:1027E000005CD8B416EF25F00B0E035C05E1C60EB5
:1027F000005CD8B49DEF25F00B0E035C05E1C70E1D
:10280000005CD8B41DEF26F00B0E035C05E1C80E8A
:10281000005CD8B47CEF26F00F0E035C05E1A00E3F
:10282000005CD8B440EF27F00F0E035C05E1A10E69
:10283000005CD8B47AEF27F00F0E035C05E1A20E1E
:10284000005CD8B47AEF27F00F0E035C05E1A30E0D
:10285000005CD8B47AEF27F00F0E035C05E1A40EFC
:10286000005CD8B47AEF27F00F0E035C05E1A50EEB
:10287000005CD8B47AEF27F00F0E035C05E1A60EDA
:10288000005CD8B4DFEF27F00F0E035C05E1A70E64
:10289000005CD8B444EF28F0130E035C05E1880E09
:1028A000005CD8B424EF2AF0130E035C05E1890E16
:1028B000005CD8B4BEEF2AF0C9EF2AF00101776BB3
:1028C000786B0001D6EC08F01C0EF66E060EF76E63
:1028D00009EC09F019EC09F0010E0101776F786B32
:1028E0000001D6EC08F0280EF66E060EF76E09EC25
:1028F00009F019EC09F0020E0101776F786B000105
:10290000D6EC08F019EC09F0010E0101756F110EFB
:10291000746F766B000165EC09F0CBEF2AF00101D2
:10292000776B786B0001D6EC08F0340EF66E060E6D
:10293000F76E09EC09F05DC074F1130E0101756FBB
:102940000001E3EC0BF0DF0E01017F6F0001E0EC12
:1029500008F0430E01017F6F0001E0EC08F019EC74
:1029600009F0010E0101776F786B0001D6EC08F0D9
:102970003C0EF66E060EF76E09EC09F05EC074F1BF
:10298000130E0101756F0001E3EC0BF0DF0E010186
:102990007F6F0001E0EC08F0430E01017F6F000142
:1029A000E0EC08F019EC09F0020E0101776F786B8A
:1029B0000001D6EC08F019EC09F01EA613D00101B5
:1029C000756B746B766B000165EC09F0515202E196
:1029D000010E536E51A605D0535203E0FE6BFD6B02
:1029E000536A08D0110E0101756F746B766B00018C
:1029F00065EC09F0CBEF2AF05352D8A4ABD0010E0E
:102A0000536E0101776B786B0001D6EC08F0010181
:102A1000746B766B756B000141EC0CF0440EF66E36
:102A2000060EF76E09EC09F0000EE96E6AC077F148
:102A300069C076F134EC0DF03A0E01017F6F0001B0
:102A4000E0EC08F029C076F1010E0101776F00017A
:102A500097EC0DF03A0E01017F6F0001E0EC08F0F9
:102A60002AC076F1010E0101776F000197EC0DF09D
:102A7000010E0101776F786B0001D6EC08F0040EAF
:102A80000101746F766B756B000141EC0CF04A0E1E
:102A9000F66E060EF76E09EC09F0000EE96E6AC0DC
:102AA00077F169C076F134EC0DF03A0E01017F6FD9
:102AB0000001E0EC08F029C076F1010E0101776F0A
:102AC000000197EC0DF03A0E01017F6F0001E0EC80
:102AD00008F02AC076F1010E0101776F000197EC32
:102AE0000DF0020E0101776F786B0001D6EC08F053
:102AF000080E0101746F766B756B000141EC0CF0F0
:102B0000500EF66E060EF76E09EC09F0000EE96E37
:102B10006AC077F169C076F134EC0DF03A0E01012C
:102B20007F6F0001E0EC08F029C076F1010E010191
:102B3000776F000197EC0DF03A0E01017F6F0001F5
:102B4000E0EC08F02AC076F1010E0101776F000178
:102B500097EC0DF01EA614D00101756B746B766BAB
:102B6000000165EC09F0515202E1020E536E51A4CE
:102B700006D05350020803E1FE6BFD6B536A08D088
:102B8000110E0101756F746B766B000165EC09F035
:102B9000FD51EA0803E1FE51030801E0536ACBEF5F
:102BA0002AF00101776B786B0001D6EC08F0560E25
:102BB000F66E060EF76E09EC09F019EC09F0010E3D
:102BC0000101776F786B0001D6EC08F05E0EF66EAF
:102BD000060EF76E09EC09F019EC09F0020E01017E
:102BE000776F786B0001D6EC08F019EC09F0110E44
:102BF0000101756F400E746F766B000165EC09F092
:102C000001C062F0625303E0FE6BFD6B1D8CCBEFE5
:102C10002AF00101776B786B0001D6EC08F0640EA6
:102C2000F66E060EF76E09EC09F0010E0101776FE2
:102C3000786B0001D6EC08F019EC09F0020E0101E6
:102C4000776F786B0001D6EC08F019EC09F01EA63E
:102C50000BD00101756B400E746F766B000165EC53
:102C600009F001C062F00BD0110E0101756F400E2A
:102C7000746F766B000165EC09F001C062F062537D
:102C800007E0FE6BFD6B1D928CC08EF08BC08DF04B
:102C9000CBEF2AF00101776B786B0001D6EC08F0DE
:102CA000760EF66E060EF76E09EC09F019EC09F0D7
:102CB000010E0101776F786B0001D6EC08F0860EEB
:102CC000F66E060EF76E09EC09F019EC09F0020E2B
:102CD0000101776F786B0001D6EC08F0900EF66E6C
:102CE000060EF76E09EC09F0200E01017F6F00015E
:102CF000E0EC08F0460E01017F6F0001E0EC08F007
:102D0000100EE96E090E0101776FDA0E766F000181
:102D100034EC0DF019EC09F0110E0101756F746BB4
:102D2000766B000165EC09F0CBEF2AF00101776BBF
:102D3000786B0001D6EC08F09A0EF66E060EF76E70
:102D400009EC09F019EC09F0010E0101776F786BBD
:102D50000001D6EC08F0A20EF66E060EF76E09EC36
:102D600009F019EC09F0020E0101776F786B000190
:102D7000D6EC08F019EC09F0110E0101756F400E48
:102D8000746F766B000165EC09F001C062F062536C
:102D900001E0FF00CBEF2AF0010164A34FD0776B75
:102DA000786B0001D6EC08F0A80EF66E060EF76EF2
:102DB00009EC09F019EC09F0010E0101776F786B4D
:102DC0000001D6EC08F0B20EF66E060EF76E09ECB6
:102DD00009F019EC09F0020E0101776F786B000120
:102DE000D6EC08F05B0E01017F6F0001E0EC08F00B
:102DF000200E01017F6F0001E0EC08F0100EE96E7B
:102E000084C077F183C076F134EC0DF0C30EF66E1A
:102E1000060EF76E060E0101766F0001D8EC0DF07C
:102E200019EC09F0110E0101756F746B766B0001DE
:102E300065EC09F001C062F006D00101030E00014B
:102E4000FE6FEE0EFD6FCBEF2AF00101776B786B12
:102E50000001D6EC08F0CA0EF66E060EF76E09EC0D
:102E600009F019EC09F0010E0101776F786B000190
:102E7000D6EC08F0DA0EF66E060EF76E09EC09F0E5
:102E800063C074F1130E0101756F0001E3EC0BF0E8
:102E9000DF0E01017F6F0001E0EC08F0430E01013D
:102EA0007F6F0001E0EC08F019EC09F0020E01015F
:102EB000776F786B0001D6EC08F0E20EF66E060E26
:102EC000F76E09EC09F064C074F1130E0101756F1F
:102ED0000001E3EC0BF0DF0E01017F6F0001E0EC7D
:102EE00008F0430E01017F6F0001E0EC08F019ECDF
:102EF00009F0100E0101756F746B766B000165ECC3
:102F000009F0CBEF2AF0216A0101776B786B0001A1
:102F1000D6EC08F0EA0EF66E060EF76E09EC09F034
:102F2000010E0101776F786B0001D6EC08F019EC07
:102F300009F0020E0101776F786B0001D6EC08F002
:102F400019EC09F0010E0101756F110E746F766BAB
:102F5000000165EC09F0CBEF2AF0010164A102D079
:102F6000050E216E776B786B0001D6EC08F0FC0E35
:102F7000F66E060EF76E09EC09F019EC09F0010E79
:102F80000101776F786B0001D6EC08F0080EF66E41
:102F9000070EF76E09EC09F0010EE96E1EC177F11C
:102FA0001DC176F134EC0DF019EC09F0020E0101AF
:102FB000776F786B0001D6EC08F0160EF66E070EF0
:102FC000F76E09EC09F0120EF66E070EF76E030E9F
:102FD0000101766F0001D8EC0DF019EC09F0110E2B
:102FE0000101756F746B766B000165EC09F001C02F
:102FF00062F0CBEF2AF00101776B786B0001D6EC21
:1030000008F01C0EF66E070EF76E09EC09F019ECCD
:1030100009F0010E0101776F786B0001D6EC08F022
:10302000020E0101746F0001EDEC0DF019EC09F0D6
:10303000020E0101776F786B0001D6EC08F0280EC4
:10304000F66E070EF76E09EC09F019EC09F0110E97
:103050000101756F330E746F766B000165EC09F03A
:1030600001C062F062BF05D06251000802E28186B1
:1030700003D062AF01D08196CBEF2AF00101776BCC
:10308000786B0001D6EC08F0380EF66E070EF76E7E
:1030900009EC09F019EC09F0010E0101776F786B6A
:1030A0000001D6EC08F0030E0101746F0001EDEC95
:1030B0000DF019EC09F0020E0101776F786B000139
:1030C000D6EC08F0440EF66E070EF76E09EC09F028
:1030D00019EC09F0110E0101756F330E746F766BE8
:1030E000000165EC09F001C062F062BF05D06251D9
:1030F000000802E2828003D062AF01D08290CBEF61
:103100002AF00101776B786B0001D6EC08F0540EC1
:10311000F66E070EF76E09EC09F019EC09F0010ED6
:103120000101776F786B0001D6EC08F0060E010103
:10313000746F0001EDEC0DF019EC09F0020E0101C5
:10314000776F786B0001D6EC08F05A0EF66E070E1A
:10315000F76E09EC09F019EC09F0110E0101756F19
:10316000330E746F766B000165EC09F001C062F0FC
:1031700062BF05D06251000802E2828403D062AFD0
:1031800001D08294CBEF2AF00101776B786B0001BC
:10319000D6EC08F06A0EF66E070EF76E09EC09F031
:1031A00019EC09F0010E0101776F786B0001D6EC84
:1031B00008F0070E0101746F0001EDEC0DF019EC41
:1031C00009F0020E0101776F786B0001D6EC08F070
:1031D000780EF66E070EF76E09EC09F019EC09F09F
:1031E000110E0101756F330E746F766B000165EC83
:1031F00009F001C062F062BF05D06251000802E22E
:10320000828603D062AF01D08296CBEF2AF0010113
:10321000776B786B0001D6EC08F0880EF66E070E1F
:10322000F76E09EC09F019EC09F0010E0101776F56
:10323000786B0001D6EC08F0050E0101746F0001F7
:10324000EDEC0DF019EC09F0020E0101776F786BCF
:103250000001D6EC08F0900EF66E070EF76E09EC42
:1032600009F019EC09F0110E0101756F330E746F3E
:10327000766B000165EC09F001C062F062BF05D019
:103280006251000802E2828803D062AF01D08298C6
:10329000CBEF2AF00101776B786B0001D6EC08F0D8
:1032A000A00EF66E070EF76E09EC09F019EC09F0A6
:1032B000010E0101776F786B0001D6EC08F0090E62
:1032C0000101746F0001EDEC0DF019EC09F0020E34
:1032D0000101776F786B0001D6EC08F0A80EF66E4E
:1032E000070EF76E09EC09F019EC09F0110E010157
:1032F000756F746B766B000165EC09F0CBEF2AF00B
:103300000101776B786B0001D6EC08F0B60EF66E13
:10331000070EF76E09EC09F019EC09F0010E010136
:10332000776F786B0001D6EC08F00C0E0101746F1A
:103330000001EDEC0DF019EC09F0020E0101776FC0
:10334000786B0001D6EC08F0C20EF66E070EF76E31
:1033500009EC09F019EC09F0110E0101756F746B9D
:10336000766B000165EC09F0CBEF2AF00101776B79
:10337000786B0001D6EC08F0D00EF66E070EF76EF3
:1033800009EC09F019EC09F0010E0101776F786B77
:103390000001D6EC08F00D0E0101746F0001EDEC98
:1033A0000DF019EC09F0020E0101776F786B000146
:1033B000D6EC08F0DE0EF66E070EF76E09EC09F09B
:1033C00019EC09F0110E0101756F746B766B000139
:1033D00065EC09F0CBEF2AF00101776B786B000107
:1033E000D6EC08F0EC0EF66E070EF76E09EC09F05D
:1033F00019EC09F0010E0101776F786B0001D6EC32
:1034000008F00E0E0101746F0001EDEC0DF019ECE7
:1034100009F0020E0101776F786B0001D6EC08F01D
:10342000F40EF66E070EF76E09EC09F019EC09F0D0
:10343000110E0101756F746B766B000165EC09F07C
:10344000CBEF2AF0030E0101746F6CC076F16BC0F4
:1034500075F1776B0001D1EC06F002C06CF001C091
:103460006BF00101776B786B0001D6EC08F0020E6F
:10347000F66E080EF76E09EC09F0010EE96E6CC0ED
:1034800077F16BC076F134EC0DF019EC09F0010E18
:103490000101776F786B0001D6EC08F019EC09F0A8
:1034A000020E0101776F786B0001D6EC08F00A0E6E
:1034B000F66E080EF76E09EC09F019EC09F0110E22
:1034C0000101756F746B766B000165EC09F0CBEF51
:1034D0002AF0070E0101746F6EC076F16DC075F1B0
:1034E000776B0001D1EC06F002C06EF001C06DF008
:1034F0000101776B786B0001D6EC08F01A0EF66EBE
:10350000080EF76E09EC09F0010EE96E6EC077F156
:103510006DC076F134EC0DF019EC09F0010E0101EB
:10352000776F786B0001D6EC08F019EC09F0020E09
:103530000101776F786B0001D6EC08F0220EF66E71
:10354000080EF76E09EC09F019EC09F0110E0101F3
:10355000756F746B766B000165EC09F0CBEF2AF0A8
:103560000B0E0101746F70C076F16FC075F1776B4F
:103570000001D1EC06F002C070F001C06FF0010153
:10358000776B786B0001D6EC08F0320EF66E080E01
:10359000F76E09EC09F0010EE96E70C077F16FC0AB
:1035A00076F134EC0DF019EC09F0010E0101776FA2
:1035B000786B0001D6EC08F019EC09F0020E01015D
:1035C000776F786B0001D6EC08F03A0EF66E080EB5
:1035D000F76E09EC09F019EC09F0110E0101756F95
:1035E000746B766B000165EC09F0CBEF2AF00F0EDF
:1035F0000101746F72C076F171C075F1776B0001D3
:10360000D1EC06F002C072F001C071F00101776BDD
:10361000786B0001D6EC08F04A0EF66E080EF76ED5
:1036200009EC09F0010EE96E72C077F171C076F114
:1036300034EC0DF019EC09F0010E0101776F786B95
:103640000001D6EC08F019EC09F0020E0101776FC9
:10365000786B0001D6EC08F0520EF66E080EF76E8D
:1036600009EC09F019EC09F0110E0101756F746B8A
:10367000766B000165EC09F0CBEF2AF0130E010127
:10368000746F74C076F173C075F1776B0001D1EC83
:1036900006F002C074F001C073F00101776B786B23
:1036A0000001D6EC08F0640EF66E080EF76E09EC19
:1036B00009F0010EE96E74C077F173C076F134EC55
:1036C0000DF019EC09F0010E0101776F786B000124
:1036D000D6EC08F019EC09F0020E0101776F786B57
:1036E0000001D6EC08F06C0EF66E080EF76E09ECD1
:1036F00009F019EC09F0110E0101756F746B766B0E
:10370000000165EC09F0CBEF2AF00101776B786BD3
:103710000001D6EC08F07E0EF66E080EF76E09EC8E
:1037200009F019EC09F0010E0101776F786B0001C7
:10373000D6EC08F0880EF66E080EF76E09EC09F06C
:1037400019EC09F0535215E1010E536E6C5311E15F
:103750006B5103080EE381BC0CD0010164BF02D0A1
:10376000000107D01EA402D0000103D0020E536E48
:103770000001020E0101776F786B0001D6EC08F0B2
:103780005350020807E1960EF66E080EF76E09EC2C
:1037900009F006D0A20EF66E080EF76E09EC09F0DD
:1037A00019EC09F0110E0101756F400E746F766B04
:1037B000000165EC09F001C062F0625311E0535062
:1037C00002080EE1040E216E010E306E8A6B896BC9
:1037D00092EC07F07A6B796BFE6BFD6B92EC07F065
:1037E000FD51E00803E1FE51070801E0536ACBEF09
:1037F0002AF00101776B786B0001D6EC08F0B00E6F
:10380000F66E080EF76E09EC09F019EC09F0110ECE
:103810000101756F220E746F766B000165EC09F083
:1038200001C062F0535205E1010E536E686B676B85
:10383000626F6253D8B47DD0036A6251E8BE03065A
:1038400067270350682368AF02D0686B676B68BF57
:1038500008D0685303E167517F0803E2686B7F0E6D
:10386000676F67C020F0D8902034306E010E0101E0
:10387000776F786B0001D6EC08F07E0E30240101E2
:10388000746F816F010E826F000135EC06F002C08B
:1038900075F101C074F1CC0EF66E080EF76E09ECEE
:1038A00009F020C076F1110E0101776F000197EC4D
:1038B0000DF0220E01017F6F0001E0EC08F0000E18
:1038C000E96E75C177F174C176F134EC0DF0C60E76
:1038D000F66E080EF76E040E0101766F0001D8EC4B
:1038E0000DF0020E0101776F786B0001D6EC08F045
:1038F000010E205C006ED89000360050036A8F0FD6
:10390000E96E000E0320EA6EECCF75F1ED52EFCFB9
:1039100074F1D20EF66E080EF76E09EC09F0000E87
:10392000E96E75C177F174C176F134EC0DF019ECE4
:1039300009F0FD51E10803E1FE51070801E0536A77
:10394000CBEF2AF00101776B786B0001D6EC08F021
:10395000D80EF66E080EF76E09EC09F019EC09F0B6
:10396000010E0101776F786B0001D6EC08F00A0EAA
:103970000101746F0001EDEC0DF019EC09F0020E7D
:103980000101776F786B0001D6EC08F0E00EF66E5F
:10399000080EF76E09EC09F019EC09F0110E01019F
:1039A000756F746B766B000165EC09F0CBEF2AF054
:1039B0000101776B786B0001D6EC08F0EE0EF66E25
:1039C000080EF76E09EC09F019EC09F0010E01017F
:1039D000776F786B0001D6EC08F00B0E0101746F65
:1039E0000001EDEC0DF019EC09F0020E0101776F0A
:1039F000786B0001D6EC08F0F60EF66E080EF76E46
:103A000009EC09F019EC09F0110E0101756F746BE6
:103A1000766B000165EC09F0CBEF2AF00101776BC2
:103A2000786B0001D6EC08F0040EF66E090EF76E06
:103A300009EC09F019EC09F0010E0101776F786BC0
:103A40000001D6EC08F0040E0101746F0001EDECEA
:103A50000DF019EC09F0020E0101776F786B00018F
:103A6000D6EC08F0120EF66E090EF76E09EC09F0AE
:103A700019EC09F0110E0101756F330E746F766B3E
:103A8000000165EC09F001C062F062BF05D062512F
:103A9000000802E2828A03D062AF01D0829ACBEFA3
:103AA0002AF00101776B786B0001D6EC08F0220E4A
:103AB000F66E090EF76E09EC09F019EC09F0010E2B
:103AC0000101776F786B0001D6EC08F0080E010158
:103AD000746F0001EDEC0DF019EC09F0020E01011C
:103AE000776F786B0001D6EC08F02A0EF66E090E9F
:103AF000F76E09EC09F019EC09F0100E0101756F71
:103B0000330E746F766B000165EC09F001C062F052
:103B100062BF05D06251000802E2808803D062AF24
:103B200001D08098CBEF2AF00101776B786B000110
:103B3000D6EC08F03A0EF66E090EF76E09EC09F0B5
:103B400019EC09F0010E0101776F786B0001D6ECDA
:103B500008F019EC09F0020E0101776F786B000193
:103B6000D6EC08F019EC09F0010E0101756F110E89
:103B7000746F766B000165EC09F0CBEF2AF0010160
:103B8000776B786B0001D6EC08F0440EF66E090EE8
:103B9000F76E09EC09F019EC09F0010E0101776FDD
:103BA000786B0001D6EC08F05B0E01017F6F00011D
:103BB000E0EC08F05BC076F1180E0101776F0001B0
:103BC00097EC0DF03A0E01017F6F0001E0EC08F078
:103BD00033C076F1130E0101776F000197EC0DF001
:103BE0005D0E01017F6F0001E0EC08F019EC09F0B7
:103BF000020E0101776F786B0001D6EC08F04C0ED5
:103C0000F66E090EF76E040E0101766F0001D8EC16
:103C10000DF0000EE96E8AC077F189C076F134ECC0
:103C20000DF019EC09F053520DE1480E0101816FBE
:103C3000826B000135EC06F002C068F001C067F04D
:103C4000010E536E110E0101756F220E746F010E7D
:103C5000766F000165EC09F001C062F0625309E083
:103C6000020E536E036A6251E8BE030667270350D3
:103C7000682368AF07D05B50010802E2D8905B323E
:103C8000686B676968BF0AD06851000807E25B503B
:103C9000040802E3D8905B36686B676B67C033F04B
:103CA000FD51B90803E1FE510B0818E0535002081A
:103CB00014E1480E01017A6F7C6B67C07BF17D6B6C
:103CC000000165EC06F04E0E01017A6F7C6B5BC063
:103CD0007BF17D6B000165EC06F0536ACBEF2AF0B7
:103CE0000101776B786B0001D6EC08F0560EF66E8A
:103CF000090EF76E09EC09F019EC09F0010E01014B
:103D0000776F786B0001D6EC08F0640EF66E090E42
:103D1000F76E040E0101766F0001D8EC0DF0020E73
:103D2000E96EFCC077F1FBC076F134EC0DF06C0E5F
:103D3000F66E090EF76E050E0101766F0001D8ECE4
:103D40000DF0010EE96E6CC077F16BC076F134ECCA
:103D50000DF0020E0101776F786B0001D6EC08F0D0
:103D60005350020806E1760EF66E090EF76E09EC66
:103D700009F0535216E1880EF66E090EF76E09EC43
:103D800009F0010EE96EFCC077F1FBC076F134EC6E
:103D90000DF0FB516B27FC516C23FC6BFB6B010E90
:103DA000536E535002080BE1140E0101756F746BD2
:103DB000766B000165EC09F001C062F00BD0110ECA
:103DC0000101756F400E746F766B000165EC09F0B0
:103DD00001C062F0625326E0020E536EFC6BFB6B77
:103DE000030E0101746F6CC076F16BC075F1776BD7
:103DF0000001D1EC06F002C06CF001C06BF0020EC5
:103E00000101746F960E756F000120EC06F0010140
:103E1000742FF8D76CC0FCF06BC0FBF000016C6B2A
:103E2000050E6B6FFD51BA0803E1FE510B0829E046
:103E30005350020819E1010164B102D0000114D00D
:103E40000001FD51BB0810E1FE510B080DE1600EB1
:103E500001017A6FFCC07CF1FBC07BF1010E7D6F2C
:103E6000000165EC06F00CD0600E0101816F010EBF
:103E7000826F000135EC06F002C0FCF001C0FBF0DF
:103E8000536ACBEF2AF00101776B786B0001D6EC17
:103E900008F0960EF66E090EF76E09EC09F019ECB3
:103EA00009F0010E0101776F786B0001D6EC08F084
:103EB000A40EF66E090EF76E040E0101766F000176
:103EC000D8EC0DF032C076F1130E0101776F0001CE
:103ED00097EC0DF0AB0EF66E090EF76E050E0101B4
:103EE000766F0001D8EC0DF0010EE96E6EC077F12F
:103EF0006DC076F134EC0DF0020E0101776F786B36
:103F00000001D6EC08F05350020806E1B60EF66E3A
:103F1000090EF76E09EC09F0535215E1C80EF66E62
:103F2000090EF76E09EC09F032C076F1130E0101AB
:103F3000776F000197EC0DF032506D27000E6E2365
:103F4000326A010E536E535002080BE1140E010148
:103F5000756F746B766B000165EC09F001C062F05F
:103F60000BD0110E0101756F400E746F766B00015E
:103F700065EC09F001C062F0625323E0020E536E5B
:103F8000326A070E0101746F6EC076F16DC075F173
:103F9000776B0001D1EC06F002C06EF001C06DF04D
:103FA000020E0101746F960E756F000120EC06F091
:103FB0000101742FF8D76DC032F000016E6B050E51
:103FC0006D6FFD51BB0803E1FE510B0824E0535017
:103FD000020817E1010164B102D0000112D0000112
:103FE000FD51BC080EE1FE510B080BE1460E01012C
:103FF0007A6F7C6B32C07BF17D6B000165EC06F063
:1040000009D0460E0101816F826B000135EC06F08C
:1040100001C032F0536ACBEF2AF00101776B786B65
:104020000001D6EC08F0D60EF66E090EF76E09EC1C
:1040300009F019EC09F0010E0101776F786B0001AE
:10404000D6EC08F0E20EF66E090EF76E09EC09F0F8
:10405000000EE96E68C077F167C076F134EC0DF0C0
:1040600019EC09F0020E0101776F786B0001D6ECB4
:1040700008F019EC09F053520EE10C0E0101816FAA
:10408000010E826F000135EC06F002C068F001C03D
:1040900067F0010E536E110E0101756F220E746FE1
:1040A000020E766F000165EC09F001C062F0625308
:1040B00010E0020E536E62BF08D06251000805E2A4
:1040C000320E6727000E682304D0320E675F000EA1
:1040D000685B68AF02D0686B676B68BF0CD06851D3
:1040E0004D0809E2FF0A03E16751200804E24E0E81
:1040F000686F200E676FFD51BC0803E1FE510B088D
:1041000014E05350020810E1010164BF02D0000125
:104110000BD00C0E7A6F68C07CF167C07BF1010E8A
:104120007D6F000165EC06F0536ACBEF2AF00101C8
:10413000776B786B0001D6EC08F0EA0EF66E090E8C
:10414000F76E09EC09F019EC09F0010E0101776F27
:10415000786B0001D6EC08F0F40EF66E090EF76EDF
:1041600009EC09F067C076F1110E0101776F0001CB
:1041700097EC0DF019EC09F0020E0101776F786BE6
:104180000001D6EC08F019EC09F053520DE1490E8C
:104190000101816F826B000135EC06F002C068F00E
:1041A00001C067F0010E536E110E0101756F220EF2
:1041B000746F010E766F000165EC09F001C062F0CA
:1041C000625309E0020E536E036A6251E8BE0306B1
:1041D00067270350682368AF02D0686B676B68BFBE
:1041E00008D0685303E16751630803E2686B630E0C
:1041F000676FFD51BD0803E1FE510B0816E05350F7
:10420000020810E101016451030BD8A402D000019F
:1042100009D0490E7A6F7C6B67C07BF17D6B000122
:1042200065EC06F067C061F0536ACBEF2AF001013C
:10423000776B786B0001D6EC08F0FC0EF66E090E79
:10424000F76E09EC09F019EC09F0010E0101776F26
:10425000786B0001D6EC08F0080EF66E0A0EF76EC9
:1042600009EC09F0010EE96E68C077F167C076F1DC
:1042700034EC0DF019EC09F0020E0101776F786B48
:104280000001D6EC08F019EC09F053520EE1620E71
:104290000101816F010E826F000135EC06F002C052
:1042A00068F001C067F0010E536E110E0101756FC9
:1042B000220E746F766B000165EC09F001C062F0AC
:1042C000625310E0020E536E62BF08D062510008C4
:1042D00005E2640E6727000E682304D0640E675F52
:1042E000000E685B68BF07D06851765D08E303E1A4
:1042F0007551675D04E276C068F075C067F068BF0D
:104300000CD06851120809E2FF0A03E167518808DE
:1043100004E2130E686F880E676FFD51BE0803E15B
:10432000FE510B0814E0535002080CE1620E01012B
:104330007A6F68C07CF167C07BF1010E7D6F000170
:1043400065EC06F068C00EF167C00DF1536ACBEF63
:104350002AF01EB206D00B0EFE6FC50EFD6FCBEF1E
:104360002AF00101776B786B0001D6EC08F0100E93
:10437000F66E0A0EF76E09EC09F019EC09F0010E61
:104380000101776F786B0001D6EC08F0180EF66E1D
:104390000A0EF76E09EC09F067C076F1110E010103
:1043A000776F000197EC0DF019EC09F0020E010196
:1043B000776F786B0001D6EC08F019EC09F05352D6
:1043C0000DE1310E0101816F826B000135EC06F0C9
:1043D00002C068F001C067F0010E536E110E0101BA
:1043E000756F220E746F010E766F000165EC09F097
:1043F00001C062F062531FE0020E536E036A625105
:10440000E8BE030667270350682368BF05D06853DA
:1044100006E16751000803E3686B010E676F68BF30
:1044200008D0685303E16751640803E2686B640EC7
:10443000676F67C05CF0FD51BF0803E1FE510B08D8
:1044400012E0535002080EE1010164B102D00001F4
:1044500009D0310E7A6F7C6B67C07BF17D6B0001F8
:1044600065EC06F0536ACBEF2AF00101776B786BAD
:104470000001D6EC08F0200EF66E0A0EF76E09EC7D
:1044800009F019EC09F0010E0101776F786B00015A
:10449000D6EC08F02E0EF66E0A0EF76E09EC09F057
:1044A000010EE96E68C077F167C076F134EC0DF06B
:1044B00019EC09F0020E0101776F786B0001D6EC60
:1044C00008F019EC09F053520EE1270E0101816F3B
:1044D000010E826F000135EC06F002C068F001C0E9
:1044E00067F0010E536E110E0101756F220E746F8D
:1044F000010E766F000165EC09F001C062F06253B5
:104500001FE0020E536E036A6251E8BE030667277E
:104510000350682368AF02D0686B676B68BF0CD02C
:104520006851020809E2FF0A03E16751E80804E262
:10453000030E686FE80E676F68C014F167C013F16F
:10454000FD51C00803E1FE510B0814E0535002086E
:1045500010E1010164B102D000010BD0270E7A6F87
:1045600068C07CF167C07BF1010E7D6F000165ECD6
:1045700006F0536ACBEF2AF00101776B786B0001EC
:10458000D6EC08F0360EF66E0A0EF76E09EC09F05E
:1045900019EC09F0010E0101776F786B0001D6EC80
:1045A00008F0460EF66E0A0EF76E09EC09F0010EE1
:1045B000E96E68C077F167C076F134EC0DF019EC64
:1045C00009F0020E0101776F786B0001D6EC08F05C
:1045D0004E0EF66E0A0EF76E09EC09F0200E010180
:1045E0007F6F0001E0EC08F0340E01017F6F0001E5
:1045F000E0EC08F019EC09F053520EE1290E01012C
:10460000816F010E826F000135EC06F002C068F088
:1046100001C067F0010E536E110E0101756F220E7D
:10462000746F010E766F000165EC09F001C062F055
:1046300062531FE0020E536E036A6251E8BE030626
:1046400067270350682368AF02D0686B676B68BF49
:104650000CD06851020809E2FF0A03E16751E8083B
:1046600004E2030E686FE80E676F68C016F167C05A
:1046700015F1FD51C10803E1FE510B0814E0535040
:10468000020810E1010164B102D000010BD0290E33
:104690007A6F68C07CF167C07BF1010E7D6F00010D
:1046A00065EC06F0536ACBEF2AF00101776B786B6B
:1046B0000001D6EC08F0540EF66E0A0EF76E09EC07
:1046C00009F019EC09F0010E0101776F786B000118
:1046D000D6EC08F0640EF66E0A0EF76E09EC09F0DF
:1046E000010EE96E68C077F167C076F134EC0DF029
:1046F00019EC09F0020E0101776F786B0001D6EC1E
:1047000008F06C0EF66E0A0EF76E09EC09F0200E3A
:1047100001017F6F0001E0EC08F0350E01017F6FB1
:104720000001E0EC08F019EC09F053520EE12B0EF9
:104730000101816F010E826F000135EC06F002C0AD
:1047400068F001C067F0010E536E110E0101756F24
:10475000220E746F010E766F000165EC09F001C046
:1047600062F062531FE0020E536E036A6251E8BEAC
:10477000030667270350682368AF02D0686B676B36
:1047800068BF0CD06851020809E2FF0A03E16751D3
:10479000E80804E2030E686FE80E676F68C018F15E
:1047A00067C017F1FD51C20803E1FE510B0814E088
:1047B0005350020810E1010164B102D000010BD096
:1047C0002B0E7A6F68C07CF167C07BF1010E7D6FA4
:1047D000000165EC06F0536ACBEF2AF00101776B1C
:1047E000786B0001D6EC08F0720EF66E0A0EF76ECA
:1047F00009EC09F019EC09F0010E0101776F786BF3
:104800000001D6EC08F07C0EF66E0A0EF76E09EC8D
:1048100009F0010EE96E68C077F167C076F134ECFB
:104820000DF019EC09F0020E0101776F786B0001B1
:10483000D6EC08F019EC09F053520EE12D0E0101EF
:10484000816F010E826F000135EC06F002C068F046
:1048500001C067F0010E536E110E0101756F220E3B
:10486000746F010E766F000165EC09F001C062F013
:1048700062531FE0020E536E036A6251E8BE0306E4
:1048800067270350682368AF02D0686B676B68BF07
:104890000CD06851020809E2FF0A03E16751E808F9
:1048A00004E2030E686FE80E676F68C01AF167C014
:1048B00019F1FD51C30803E1FE510B0814E05350F8
:1048C000020810E1010164B102D000010BD02D0EED
:1048D0007A6F68C07CF167C07BF1010E7D6F0001CB
:1048E00065EC06F0536ACBEF2AF01EB206D00B0E31
:1048F000FE6FBE0EFD6FCBEF2AF00101776B786B78
:104900000001D6EC08F0840EF66E0A0EF76E09EC84
:1049100009F019EC09F0010E0101776F786B0001C5
:10492000D6EC08F0900EF66E0A0EF76E09EC09F060
:10493000010EE96E68C077F167C076F134EC0DF0D6
:1049400019EC09F0020E0101776F786B0001D6ECCB
:1049500008F0980EF66E0A0EF76E09EC09F0200EBC
:1049600001017F6F0001E0EC08F0330E01017F6F61
:104970000001E0EC08F019EC09F053520EE12F0EA3
:104980000101816F010E826F000135EC06F002C05B
:1049900068F001C067F0010E536E110E0101756FD2
:1049A000220E746F010E766F000165EC09F001C0F4
:1049B00062F062531FE0020E536E036A6251E8BE5A
:1049C000030667270350682368AF02D0686B676BE4
:1049D00068BF0CD06851020809E2FF0A03E1675181
:1049E000E80804E2030E686FE80E676F68C01CF108
:1049F00067C01BF1FD51C40803E1FE510B0814E030
:104A00005350020810E1010164B102D000010BD043
:104A10002F0E7A6F68C07CF167C07BF1010E7D6F4D
:104A2000000165EC06F0536ACBEF2AF00101776BC9
:104A3000786B0001D6EC08F09E0EF66E0A0EF76E4B
:104A400009EC09F019EC09F0010E0101776F786BA0
:104A50000001D6EC08F067C076F1110E0101776F06
:104A6000000197EC0DF0AF0EF66E0A0EF76E090E10
:104A70000101766F0001D8EC0DF019EC09F0020E7F
:104A80000101776F786B0001D6EC08F019EC09F0A2
:104A900053520DE1410E0101816F826B000135EC33
:104AA00006F002C068F001C067F0010E536E110EEF
:104AB0000101756F220E746F010E766F000165ECB7
:104AC00009F001C062F0625309E0020E536E036AFE
:104AD0006251E8BE030667270350682368AF02D01F
:104AE000686B676B68BF08D0685303E16751630860
:104AF00003E2686B630E676FFD51C50803E1FE5169
:104B00000B0819E0535002080EE1010164B102D014
:104B1000000109D0410E7A6F7C6B67C07BF17D6B21
:104B2000000165EC06F067C02EF02E5202E01C8AF0
:104B300001D01C9A536ACBEF2AF00101776B786B96
:104B40000001D6EC08F0BA0EF66E0A0EF76E09EC0C
:104B500009F019EC09F0010E0101776F786B000183
:104B6000D6EC08F0C60EF66E0A0EF76E09EC09F0E8
:104B700067C076F1110E0101776F000197EC0DF01F
:104B800019EC09F0020E0101776F786B0001D6EC89
:104B900008F019EC09F053520DE1420E0101816F4A
:104BA000826B000135EC06F002C068F001C067F0CE
:104BB000010E536E110E0101756F220E746F010EFE
:104BC000766F000165EC09F001C062F0625309E004
:104BD000020E536E036A6251E8BE03066727035054
:104BE000682368AF02D0686B676B68BF08D06853F2
:104BF00003E16751630803E2686B630E676FFD5161
:104C0000C60803E1FE510B0816E0535002080EE1FE
:104C1000010164B102D0000109D0420E7A6F7C6BB1
:104C200067C07BF17D6B000165EC06F067C02FF07B
:104C3000536A686B676BCBEF2AF00101776B786B77
:104C40000001D6EC08F0CE0EF66E0A0EF76E09ECF7
:104C500009F05B0E01017F6F0001E0EC08F067C016
:104C600076F1130E0101776F000197EC0DF05D0EE8
:104C700001017F6F0001E0EC08F019EC09F0010E72
:104C80000101776F786B0001D6EC08F019EC09F0A0
:104C9000020E0101776F786B0001D6EC08F019EC79
:104CA00009F0110E0101756F220E746F010E766FFF
:104CB000000165EC09F001C062F0625307E0036A8D
:104CC0006251E8BE030667270350682368AF02D02D
:104CD000686B676B68BF05D06851000802E2686BBB
:104CE0006769FD51C70803E1FE510B0803E0536AF1
:104CF00067C020F0CBEF2AF053523AE1010E536E19
:104D0000205224E02050040821E0205008081EE032
:104D100020500C081BE020500F0818E020504408D9
:104D200015E02050510812E0205053080FE02050A9
:104D300055080CE02050570809E02050600806E0B4
:104D40002050320803E020507F0802E21C8E01D080
:104D50001C9E000E1CBE010E0101746F20C081F16B
:104D6000826F000135EC06F002C068F001C067F008
:104D70000101776B786B0001D6EC08F0DA0EF66E65
:104D80000A0EF76E09EC09F020C076F1130E01014E
:104D9000776F000197EC0DF019EC09F0010E01019D
:104DA000776F786B0001D6EC08F019EC09F0020E71
:104DB0000101776F040E786F0001D6EC08F0DE0E6B
:104DC000F66E0A0EF76E09EC09F05B0E01017F6FBB
:104DD0000001E0EC08F0000EE96E68C077F167C0F2
:104DE00076F134EC0DF05D0E01017F6F0001E0EC17
:104DF00008F0100E0101756F220E746F010E766FB0
:104E0000000165EC09F001C062F0625309E0020E96
:104E1000536E036A6251E8BE030667270350682396
:104E200068AF02D0686B676B68BF07D06851000835
:104E300004E21CBE02D0686B6769FD51C80803E13B
:104E4000FE510B081CE05350020813E1010164BF3E
:104E500002D000010ED0000E1CBE010E746F20C0E7
:104E60007AF168C07CF167C07BF17D6F000165EC71
:104E700006F0036A20C067F003C068F0536A8BD362
:104E80000101776B786B0001D6EC08F0E40EF66E4A
:104E90000A0EF76E09EC09F019EC09F0010E010198
:104EA000776F786B0001D6EC08F019EC09F0020E70
:104EB0000101776F786B0001D6EC08F019EC09F06E
:104EC000010E546E545006080BE3036A5450640FED
:104ED000E96E010E0320EA6E300EEF6E542AF2D70F
:104EE000010E0101756F100E746F766B000165EC99
:104EF00009F051D376EC0EF0110E0101756F220E00
:104F0000746F010E766F000165EC09F001C062F06C
:104F100062BF2BD06251000828E2A00EFD5D0101A6
:104F2000746F0F0E0001FE590101756F640E742538
:104F3000E96E010E7521EA6EEF503808D8B002D044
:104F4000000113D0A00E0001FD5D0101746F0F0E72
:104F50000001FE590101756F640E7425E96E010EA2
:104F60007521EA6EEF2A29D0000162AF27D0A00E8A
:104F7000FD5D0101746F0F0E0001FE590101756F97
:104F8000640E7425E96E010E7521EA6EEF5030084B
:104F9000D8A002D0000112D0A00E0001FD5D0101D9
:104FA000746F0F0E0001FE590101756F640E7425B8
:104FB000E96E010E7521EA6EEF060001ECD276EC87
:104FC0000EF0140E0101756F220E746F010E766FD4
:104FD000000165EC09F001C062F062BF2BD06251A4
:104FE000000828E2A00EFD5D0101746F0F0E0001A4
:104FF000FE590101756F640E7425E96E010E75216D
:10500000EA6EEF503808D8B002D0000113D0A00EDD
:105010000001FD5D0101746F0F0E0001FE590101D9
:10502000756F640E7425E96E010E7521EA6EEF2A24
:1050300029D0000162AF27D0A00EFD5D0101746F81
:105040000F0E0001FE590101756F640E7425E96EA3
:10505000010E7521EA6EEF503008D8A002D0000191
:1050600012D0A00E0001FD5D0101746F0F0E000152
:10507000FE590101756F640E7425E96E010E7521EC
:10508000EA6EEF06000187D2010EEA6E6B0EE96E42
:10509000000EF3EC00F00A000900F550EE6E000976
:1050A000FBE1010E0101756F650E746F010E776FE4
:1050B0006B0E766F796B060E786F0001C8EC0EF000
:1050C000015203E1010164690001010EEA6E6B0EF9
:1050D000E96E000EFFEC00F00A000900F550EE6EDC
:1050E0000009FBE1010E0101756F650E746F010E81
:1050F000776F6B0E766F796B060E786F0001C8ECD8
:105100000EF0015204E1030E0101646F0001010E73
:10511000EA6E6B0EE96E000E0BEC01F00A0009005E
:10512000F550EE6E0009FBE1010E0101756F650E91
:10513000746F010E776F6B0E766F796B060E786F5A
:105140000001C8EC0EF0015204E1010E0101646F90
:105150000001010EEA6E6B0EE96E000E17EC01F015
:105160000A000900F550EE6E0009FBE1010E010195
:10517000756F650E746F010E776F6B0E766F796BBE
:10518000060E786F0001C8EC0EF0015233E11DAA43
:1051900010D00101643D03D000010BD00101700E5D
:1051A0007A6F7C6B7B6B7D6B000165EC06F01D9A62
:1051B0001FD01D8A832BD8B4842B1B0E01017A6F5C
:1051C00084C07CF183C07BF1010E7D6F000165EC32
:1051D00006F00101643D0BD0700E7A6F7C6B010EFE
:1051E0007B6F7D6B000165EC06F00101646B0001D3
:1051F000FE6BFD6B010EEA6E6B0EE96E000E23EC8A
:1052000001F00A000900F550EE6E0009FBE1010E05
:105210000101756F650E746F010E776F6B0E766FFF
:10522000796B060E786F0001C8EC0EF0015210E1A8
:105230004F0E01017A6F7C6B7B6B7D6B000165EC1F
:1052400006F00101646B1F901F920001FE6BFD6B65
:10525000010EEA6E6B0EE96E000E2FEC01F00A00F3
:105260000900F550EE6E0009FBE1010E0101756FBA
:10527000650E746F010E776F6B0E766F796B060E8D
:10528000786F0001C8EC0EF0015211E14F0E0101E0
:105290007A6F7C6B010E7B6F7D6B000165EC06F015
:1052A0000101646B1F801F920001FE6BFD6B010EFC
:1052B000EA6E6B0EE96E000E3BEC01F00A0009008D
:1052C000F550EE6E0009FBE1010E0101756F650EF0
:1052D000746F010E776F6B0E766F796B060E786FB9
:1052E0000001C8EC0EF0015211E14F0E01017A6F7E
:1052F0007C6B020E7B6F7D6B000165EC06F001019B
:10530000646B1F801F820001FE6BFD6B010EEA6E55
:105310006B0EE96E000E47EC01F00A000900F55033
:10532000EE6E0009FBE1010E0101756F650E746FF1
:10533000010E776F6B0E766F796B060E786F00013A
:10534000C8EC0EF0015211E14F0E01017A6F7C6B37
:10535000030E7B6F7D6B000165EC06F00101646B51
:105360001F901F820001FE6BFD6B0101645344E03E
:105370001E80776B786B0001D6EC08F0EE0EF66EAF
:105380000A0EF76E09EC09F019EC09F0010E0101A3
:10539000776F786B0001D6EC08F0FE0EF66E0A0E01
:1053A000F76E09EC09F019EC09F0020E0101776FB4
:1053B000786B0001D6EC08F0080EF66E0B0EF76E57
:1053C00009EC09F0200E01017F6F0001E0EC08F00C
:1053D000460E01017F6F0001E0EC08F0100EE96E4F
:1053E000090E0101776FDA0E766F000134EC0DF0D3
:1053F00019EC09F020D00101776B786B0001D6EC35
:1054000008F019EC09F0010E0101776F786B0001CB
:10541000D6EC08F0120EF66E0B0EF76E09EC09F0E2
:1054200019EC09F0020E0101776F786B0001D6ECE0
:1054300008F019EC09F0140E0101756F746B766BAE
:10544000000165EC09F0A7D0040E0101756F110E83
:10545000746F766B000165EC09F001C062F062BF09
:1054600014D06251000811E25650010802E3562A96
:1054700007D05650020804E15850010801E3582AA9
:105480005750030801E3572A0ED062AF0CD0565292
:1054900002E0560605D0565203E1585201E0580684
:1054A000575201E0570656C077F10101786B0001B1
:1054B000D6EC08F03D2A3D50060801E23D6A3D5019
:1054C000040807E37E0E01017F6F0001E0EC08F0A5
:1054D00006D0200E01017F6F0001E0EC08F056526B
:1054E00008E10101776B010E786F0001D6EC08F03E
:1054F00006D00101776B786B0001D6EC08F058C03C
:1055000075F10FEC0FF019EC09F0562C08D0010ED4
:105510000101776F786F0001D6EC08F007D0010E1B
:105520000101776F786B0001D6EC08F0010E58246A
:105530000101746F756F00010FEC0FF019EC09F0A9
:105540005650020809E1020E0101776F010E786FD3
:105550000001D6EC08F007D0020E0101776F786BDE
:105560000001D6EC08F0020E58240101746F756F2B
:1055700000010FEC0FF019EC09F00DD057500408A2
:1055800001E11E8A5750000801E21D8CFE6BFD6B85
:1055900002D0FE6BFD6B5AD0FD51FE1157E11DA6E6
:1055A00055D01D961DAE04D0515201E11D9E4ED026
:1055B00051524CE0512C02D0050E596E5150020848
:1055C0000BE1030EFE6FEC0EFD6F1D8E0101006BF3
:1055D000A00E0001FF6F1E8651500F080CE1030E54
:1055E000FE6FE80EFD6F1D8E0101006B0001FF6B69
:1055F000536A1E96576A515004080BE1030EFE6F62
:10560000EA0EFD6F1D8E0101006B0001FF6B536AF6
:105610001E86515008080BE1030EFE6FE90EFD6F68
:105620001D8E0101006B0001FF6B536A1E865150F5
:105630000C080CE1130EFE6F880EFD6F1D8E01012C
:10564000006B0001FF6B576A586A566A21500AE0E6
:10565000040AD8B46DEF31F0010AD8B4CFEF32F0BC
:10566000D2EF32F01CA8AAD11C98030E0101746F6E
:105670006CC076F16BC075F1010E776F0001D1EC53
:1056800006F002C06CF001C06BF0070E0101746FF0
:105690006EC076F16DC075F1010E776F0001D1EC2F
:1056A00006F002C06EF001C06DF00B0E0101746FC8
:1056B00070C076F16FC075F1010E776F0001D1EC0B
:1056C00006F002C070F001C06FF06E5303E16D513F
:1056D000F90802E26E6B6D6B6D5101010527000147
:1056E0006E510101062300016B51010107270001E2
:1056F0006C5101010823552A5550040848E2556AA7
:1057000006C17DF105C17CF17F6B050E7E6F000146
:10571000AEEC06F002C00AF101C009F10101066B0E
:10572000056B226B216B0A5303E1095103081EE24A
:105730000AC17CF109C17BF17E6B910E7D6F000186
:105740009DEC06F002C075F101C074F102C07DF15C
:1057500001C07CF101017F6B0A0E7E6F0001AEEC8F
:1057600006F002C022F101C021F1010108C17DF162
:1057700007C17CF17F6B050E7E6F0001AEEC06F079
:1057800002C00CF101C00BF10101086B076B82A68E
:1057900038D081B236D082B834D01EBE17D01E8E1B
:1057A0001CAA02D0828401D082881DA205D01D923D
:1057B0008CC08EF08BC08DF0410E816F826B00012A
:1057C00035EC06F0010E010101242E6E2E062E523C
:1057D0000AE18288400E816F826B000135EC06F091
:1057E00001C02EF0010182A80CD000017A6B796B08
:1057F00078C0F4F077C0F3F0406A1D983F6A1E9EAF
:10580000010181B202D082B605D082981E9E2E522E
:1058100001E02E0600016E5303E12F506D5D02E39F
:105820002E5203E181A201D082941EA2C7D081BE74
:1058300019D0828A1CC102F01BC101F00232013270
:1058400002320132023201C067FF02320230300BF5
:10585000006E6650CF0B0010666E20C11EF11FC196
:105860001DF1ACD081B892D082BA04D020C11EF113
:105870001FC11DF1828A81BA2DD001011E51185D10
:1058800009E303E117511D5D05E25C501D27000E81
:105890001E230BD018511E5D08E303E11D51175D57
:1058A00004E218C11EF117C11DF11EC102F01DC195
:1058B00001F00232013202320132023201C067FFCE
:1058C00002320230300B006E6650CF0B0010666E55
:1058D0005BD0000181BC2DD001011E51165D09E392
:1058E00003E115511D5D05E25C501D27000E1E23CE
:1058F0000BD016511E5D08E303E11D51155D04E256
:1059000016C11EF115C11DF11EC102F01DC101F02D
:105910000232013202320132023201C067FF02322A
:105920000230300B006E6650CF0B0010666E2CD02C
:10593000000101011E511A5D09E303E119511D5DCA
:1059400005E25C501D27000E1E230BD01A511E5D70
:1059500008E303E11D51195D04E21AC11EF119C1EA
:105960001DF11EC102F01DC101F0023201320232EE
:105970000132023201C067FF02320230300B006E8A
:105980006650CF0B0010666E1AD00001829A14C1C7
:105990001EF113C11DF11EC102F01DC101F0023242
:1059A000013202320132023201C067FF023202309C
:1059B000300B006E6650CF0B0010666E01011CA606
:1059C0006CEF31F01C965A5203E04B5201E15A063B
:1059D00088C07DF187C07CF17F6B5BC07EF10001E8
:1059E000AEEC06F002C075F101C074F102C07CF1AA
:1059F00001C07BF101017E6B33C07DF100019DECA4
:105A000006F002C075F101C074F102C07DF101C061
:105A10007CF101017F6B640E7E6F0001AEEC06F03D
:105A200002C075F101C074F102C07CF101C07BF1CC
:105A300001017E6B0A0E7D6F00019DEC06F002C035
:105A40008AF001C089F0886B876B792BD8B47A2BE8
:105A50007B2BD8B47C2B7D2BD8B47E2B7F2BD8B45A
:105A6000802B3F2A1C7C595201E059060F0E010180
:105A7000746F72C076F171C075F1010E776F00011D
:105A8000D1EC06F002C072F001C071F0130E0101FA
:105A9000746F74C076F173C075F1010E776F0001F9
:105AA000D1EC06F002C074F001C073F072C075F161
:105AB00071C074F15DC076F16BEC0FF001C05DF068
:105AC00074C075F173C074F15EC076F16BEC0FF0C9
:105AD00001C05EF05EBE18D05E50310815E2645120
:105AE000800A006E5E50800A005C0EE2220E010108
:105AF0007A6F7C6B5EC07BF17BBF7C077D6B0001A6
:105B000065EC06F05EC064F06151800A006E5D5085
:105B1000800A005C01E017E21D846351800A006E78
:105B20005D50800A005C0EE21D0E01017A6F7C6BF5
:105B30005DC07BF17BBF7C077D6B000165EC06F0EF
:105B40005DC063F001D01D9426A802D01D9001D045
:105B50001D8081501C18010B0EE0006A1CB20080F1
:105B60001D500018010B07E0006A1CB4008881502A
:105B70000018100B02E1BAEF0FF001010C510308FD
:105B8000D8A0AAD004E10B51FE08D8A0A5D00001EE
:105B9000FA5101010C5DD8A09FD006E10001F95136
:105BA00001010B5DD8A098D00CC17DF10BC17CF137
:105BB000FAC07FF1F9C07EF10001AEEC06F001C041
:105BC00027F02850275CD8B081D0010E275C006EEA
:105BD000D89000360050036A8F0FE96E000E032044
:105BE000EA6EECCF75F1ED52EFCF74F1D890273417
:105BF000036A8F0FE96E000E0320EA6EECCF77F197
:105C0000ED52EFCF76F1010E275C006ED890003692
:105C10000050036A8F0FE96E000E0320EA6EECCF8E
:105C200003F0ED52EF500101765F0350775B77C1CF
:105C30007CF176C17BF17E6B0A0E7D6F00019DECDD
:105C400006F002C077F101C076F102C07DF101C01B
:105C50007CF1FAC07FF1F9C07EF1AEEC06F002C033
:105C600077F101C076F10CC17DF10BC17CF1FAC076
:105C70007FF1F9C07EF1AEEC06F000C078F103C010
:105C800079F177C17CF176C17BF103C07EF100C070
:105C90007DF100019DEC06F002C077F101C076F1C4
:105CA00002C07DF101C07CF101017F6B0A0E7E6FA5
:105CB0000001AEEC06F00150010174250001776F80
:105CC0000250010175210001786F04D082C078F084
:105CD00081C077F004D001010001786B776B7651B9
:105CE000785D05E303E17751755D01E21E8C1DB41B
:105CF00004D01EAC02D01DA80DD01DBA0BD08296C8
:105D0000FD51F00803E1FE51030803E01DA801D096
:105D10001D980AD07651785D04E305E17751755DF1
:105D200002E31DAA01D08286785101010E5D11E3C4
:105D300005E10001775101010D5D0BE303510411F1
:105D400008E0046B036B1DBA01D082961E0E416EF3
:105D500047D00351041132E078C07DF177C07CF167
:105D60007F6B640E7E6F0001AEEC06F002C075F131
:105D700001C074F102C07CF101C07BF101017E6BB6
:105D8000640E7D6F00019DEC06F002C004F101C0BD
:105D900003F1010103510001775D0101746F0451AA
:105DA000000178590101756F755303E17451320890
:105DB00004E2320E0327000E042312D02C0E0D2510
:105DC000016E010E0E21036E03500001785D09E3A0
:105DD00003E17751015C05E20101046B010E036FE1
:105DE00000011DA401D0829682A820D01DBA1ED029
:105DF00001010351041115E100017851F45D0AE33A
:105E000003E1F351775D06E278C0F4F077C0F3F078
:105E1000406A05D0402A4150405C01E31D8806D00D
:105E2000010178C0F4F077C0F3F000018B518D5D73
:105E3000006E8C518E5900C065F0666F66BF0AD047
:105E4000665303E16551000805E22B0E0101636F03
:105E50000BD0000166AF05D02D0E0101636F04D099
:105E60000001200E0101636F66C075F165C074F119
:105E7000776B0A0E766F000108EC10F002C075F126
:105E800001C074F102C003F00101015002AE08D05C
:105E9000000ED8807455006E000E7555036E0050CC
:105EA0000001F56F03C0F6F066C075F165C074F1CE
:105EB0000101776B0A0E766F000108EC10F000C04C
:105EC00074F1010103C075F103C003F0005075AF18
:105ED00008D0000ED8807455006E000E7555036E04
:105EE00000500001F76F03C0F8F0FD51FE11D8A477
:105EF000B3D10101776B786B0001D6EC08F01DA4DB
:105F00005AD0220EF66E0B0EF76E09EC09F019EC62
:105F100009F0010E0101776F786B0001D6EC08F0F3
:105F20002C0EF66E0B0EF76E09EC09F061C076F1DF
:105F3000130E0101776F000197EC0DF0DF0E0101E8
:105F40007F6F0001E0EC08F0430E01017F6F00015C
:105F5000E0EC08F0020E0101776F786B0001D6ECDF
:105F600008F0320EF66E0B0EF76E09EC09F019EC24
:105F700009F0030E0101776F786B0001D6EC08F091
:105F80003A0EF66E0B0EF76E09EC09F05DC074F177
:105F9000130E0101756F0001E3EC0BF0DF0E010140
:105FA0007F6F0001E0EC08F0430E01017F6F0001FC
:105FB000E0EC08F051D11FB019D0520EF66E0B0E66
:105FC000F76E09EC09F0000EE96E0AC177F109C11C
:105FD00076F134EC0DF04C0EF66E0B0EF76E040EEF
:105FE0000101766F0001D8EC0DF018D0660EF66E48
:105FF0000B0EF76E09EC09F0000EE96E22C177F185
:1060000021C176F134EC0DF0600EF66E0B0EF76EDA
:10601000040E0101766F0001D8EC0DF0010E0101B4
:10602000776F786B0001D6EC08F001010351041181
:1060300055E082A653D01FB21BD07A0EF66E0B0E1F
:10604000F76E000109EC09F0000EE96E04C177F16A
:1060500003C176F134EC0DF0740EF66E0B0EF76E94
:10606000040E0101766F0001D8EC0DF036D001016D
:1060700004C17CF103C17BF17E6B160E7D6F0001C4
:106080009DEC06F002C075F101C074F102C07DF113
:1060900001C07CF101017F6B640E7E6F0001AEECEC
:1060A00006F002C075F101C074F18E0EF66E0B0E93
:1060B000F76E09EC09F0000EE96E75C177F174C155
:1060C00076F134EC0DF0880EF66E0B0EF76E040EC2
:1060D0000101766F0001D8EC0DF01CD00001765163
:1060E000785D04E30AE17751755D07E37951030BAD
:1060F000006E036A0050031007E0960EF66E0B0E5A
:10610000F76E09EC09F006D0A80EF66E0B0EF76ECE
:1061100009EC09F0020E0101776F786B0001D6ECF3
:1061200008F0C60EF66E0B0EF76E09EC09F0000EC5
:10613000E96E8AC077F189C076F134EC0DF0C00EBB
:10614000F66E0B0EF76E040E0101766F0001D8ECAF
:106150000DF0030E0101776F786B0001D6EC08F0AB
:106160005A5274E01DB204D01EBA02D0595243E014
:106170008CC07DF18BC07CF101017F6B0A0E7E6FBC
:106180000001AEEC06F002C010F101C00FF18CC0AE
:106190007DF18BC07CF101017F6B0A0E7E6F0001E7
:1061A000AEEC06F000C011F1010103C012F1CE0EF9
:1061B000F66E0B0EF76E000109EC09F0020EE96EA7
:1061C00010C177F10FC176F134EC0DF02E0E010104
:1061D0007F6F0001E0EC08F0040EE96E12C177F168
:1061E00011C176F134EC0DF0D60EF66E0B0EF76E93
:1061F00009EC09F02AD0EE0EF66E0B0EF76E09ECE4
:1062000009F063C17FF1E0EC08F0020EE96EF6C020
:1062100077F1F5C076F134EC0DF02E0E01017F6FB1
:106220000001E0EC08F0040EE96EF8C077F1F7C069
:1062300076F134EC0DF0E90EF66E0B0EF76E040EEF
:106240000101766F0001D8EC0DF006D0F60EF66E67
:106250000B0EF76E09EC09F082C07DF181C07CF174
:1062600001017F6B050E7E6F0001AEEC06F002C0EF
:1062700075F101C074F178C07DF177C07CF102C086
:106280007FF101C07EF10001AEEC06F001C02DF0FF
:106290002D50FA0F20E2060FD7EF32F08290819650
:1062A0001AD01CAC81961CBC8186829014D0818649
:1062B000829011D081861CAC82901CBC82800BD055
:1062C0008280818608D081961CAC82901CBC828022
:1062D00082A001D08186010167D11CA82FD01C9813
:1062E000030E0101746F6CC076F16BC075F1010E85
:1062F000776F0001D1EC06F002C06CF001C06BF0CA
:106300006B510101072700016C5101010823552A37
:106310005550040812E2556A08C17DF107C17CF1AD
:106320007F6B050E7E6F0001AEEC06F002C00CF133
:1063300001C00BF10101086B076B00011CA62DD1F8
:106340001C96792BD8B47A2B01010C51030802E278
:106350000C6B0B6B0001FD51FE1126E10101776B07
:10636000786B0001D6EC08F0180EF66E0C0EF76E86
:1063700009EC09F0020EE96E0CC177F10BC176F160
:1063800034EC0DF00E0EF66E0C0EF76E050E0101DC
:10639000766F0001D8EC0DF0000EE96E7AC077F14F
:1063A00079C076F134EC0DF081BCC7D0010164BF37
:1063B00002D00001C2D00CC17DF10BC17CF1FAC04A
:1063C0007FF1F9C07EF10001AEEC06F001C027F0CC
:1063D0003050275CD8A0B0D0302A7AC086F079C07F
:1063E00085F0FD51FE112DE1010E0101776F786BF3
:1063F0000001D6EC08F0800E89250101746F000EB3
:1064000000018A210101756F1C0EF66E0C0EF76EED
:10641000000109EC09F0200E01017F6F0001E0ECA2
:1064200008F0010EE96E75C177F174C176F134ECB4
:106430000DF0200E01017F6F0001E0EC08F019EC77
:1064400009F0800E89250101746F000E00018A2178
:106450000101756F79C076F1F250006EF29E74C141
:10646000A9FF76C1A8FFA69CA69EA6840F01550E83
:10647000A76EAA0EA76EA682A6B2FED7A69400505B
:10648000F212810E000189250101746F000E0001D6
:106490008A210101756F7AC076F1F250006EF29E8A
:1064A00074C1A9FF76C1A8FFA69CA69EA6840F0171
:1064B000550EA76EAA0EA76EA682A6B2FED7A69408
:1064C0000050F212020E00018927000E8A23FD51AE
:1064D000FE1132E1020E0101776F786B0001D6ECFC
:1064E00008F0010E305C0101746F766F130E776F48
:1064F000000197EC0DF03A0E01017F6F0001E0EC16
:1065000008F0200E01017F6F0001E0EC08F0220E80
:10651000F66E0C0EF76E09EC09F019EC09F0030E9B
:106520000101776F786B0001D6EC08F02E0EF66E45
:106530000C0EF76E09EC09F030D0010164AF2ED0DB
:106540000F0E7A6F86C07CF185C07BF1010E7D6FE6
:10655000000165EC06F0010E305C0101746F0E0E57
:106560007A6F7C6B74C17BF17D6B000165EC06F08A
:106570007F0E01017A6F7C6B7B6B7D6B000165EC9C
:1065800006F00E0E0101816F826B000135EC06F002
:1065900001C028F092EC07F0216A010105D0010149
:1065A00003D00001216A010157EF12F00300E82433
:1065B000F76AF736C90FF66E650EF7220A00F55036
:1065C000FA6E0800F550F96E9C62A262AE62B46287
:0465D000C062C6627D
:0200000400F00A
:10000000000000000000000000000000401F000091
:1000100000000000000000000000000000180000C8
:1000200000000000000000A70158024302AA02C815
:1000300000030D02000000000000000000000000AE
:100040004B0F190000003B001E32000000000000B2
:100050000000000000000000000000000000000898
:10006000CC00DC05000000000000000000000000E3
:100070000000000000000000000000000000000080
:020000040030CA
:0E00000000E31E3F00BF850000800FE00F40B0
:00000001FF
